:020000040800F2
:100000000050002091850008D7850008D985000898
:10001000DB850008DD850008DF85000800000000A2
:10002000000000000000000000000000E185000862
:10003000E385000800000000E5850008A10800082D
:10004000EB850008ED850008EF850008F1850008C4
:10005000F3850008F5850008F7850008F985000894
:10006000FB850008FD850008FF8500080186000863
:10007000B57700080586000807860008098600088D
:100080000B8600080D8600080F8600081186000800
:1000900013860008158600081786000819860008D0
:1000A0001B8600081D8600081F86000821860008A0
:1000B000B14900082586000827860008298600081F
:1000C0002B8600082D8600082F8600083186000840
:1000D0003386000879480008693700083986000827
:1000E0003B8600083D8600083F86000810B5054C99
:1000F000237833B9044B13B10448AFF300800123D4
:10010000237010BD8003002000000000B4BD000873
:10011000084B10B51BB108490848AFF300800848E8
:10012000036803B910BD074B002BFBD0BDE810409E
:10013000184700BF0000000084030020B4BD000881
:100140008003002000000000154B002B08BF134B5C
:100150009D46A3F5803A00218B460F461348144A6A
:10016000121A08F066FC0F4B002B00D098470E4B7C
:10017000002B00D098470020002104000D000D48FE
:10018000002802D00C48AFF3008008F019FB2000D3
:10019000290004F0E5FC08F0FFFA00BF00000800A9
:1001A000005000200000000000000000800300203C
:1001B0009C140020000000000000000070B5294BD6
:1001C00086B01C681D46002C48D1684607F08AFEA0
:1001D00001A807F0EBFC4FF4004007F0BDFF012140
:1001E000112008F013F8202369461F48ADF80030AD
:1001F0008DF8034007F028FE01214FF4007008F04D
:1002000005F801264FF4602301A9184803930194CF
:100210008DF808408DF8094004948DF8146007F0BB
:10022000A1FC234632460521104807F0ECFC0F489C
:10023000314607F0C4FC0D4807F0CAFC0B4807F034
:10024000CCFC0028FAD1094807F0CBFC074807F09E
:10025000CDFC0028FAD1064B01221A6001232B6045
:1002600006B070BDA003002000080140002401403A
:100270001812002008B50121034807F0BBFC034B0E
:1002800001221A6008BD00BF002401409C03002029
:1002900038B50A4C054623680BB9002038BD022149
:1002A000074807F0FAFC0028F7D0054807F0F2FCF1
:1002B000002328802360012038BD00BF9C0300205C
:1002C000002401401723022903FB01F110B54FF070
:1002D0000903D8BF144691FBF3F1D8BF02F1FF32F6
:1002E0004FF0040392FBF3F3C8BF941E204408446C
:1002F000043018446FF0630392FBF3F318444FF497
:10030000C87392FBF3F20244072092FBF0F0C0EBBB
:10031000C000101A10BD30B50446054600202B1B46
:10032000DBB299421AD92378C3B115F8013BA3F186
:100330003002D2B2092A0DD9A3F14102052A01D80F
:10034000373B04E0A3F16102052A02D8573BDAB239
:1003500000E0002202EB001398B2E0E730BD013864
:1003600010F8013F1BB18B4208BF0270F8E77047DD
:1003700000224FF40051014807F0C2BD00100140B7
:1003800001224FF40051014807F0BABD00100140AE
:1003900007B501A807F0A6FD0121102007F036FFE0
:1003A0004FF40053ADF8043002238DF8063001A954
:1003B000102305488DF8073007F046FDFFF7E0FFF2
:1003C00003B05DF804FB00BF0010014007B501A8B1
:1003D00007F088FD0121042007F018FF4023ADF845
:1003E000043001A9482304488DF8073007F02CFD9C
:1003F00003B05DF804FB00BF0008014008B54021D0
:10040000034807F077FDB0FA80F0400908BD00BF4F
:100410000008014010B5124A034610681446E8B1BE
:10042000104A1149126864325A61104A1268013A3E
:100430001A610F4A1268DA600A68072A4FF0000250
:100440000CBF114609681A6299610A49226009685D
:1004500099600949096859600F21196010BD00BFF2
:10046000C8030020A4030020BC030020E0030020F8
:10047000A8030020D8030020B403002073B501A80E
:1004800007F030FD0121082007F0C0FE154C4FF4A5
:100490008073ADF8043004230DEB030102262046DF
:1004A0008DF807308DF8066007F0CEFC01A807F044
:1004B00019FD0121082007F0A9FE4FF40075102353
:1004C00001A920468DF80730ADF804508DF806607C
:1004D00007F0BAFC01222946204607F011FD02B0C0
:1004E00070BD00BF000C014070B5904C23682546DC
:1004F000FF2B0FD18E4A1368642B08D100224FF4D2
:1005000000718C4807F0FCFC0023236070BD0133B0
:10051000136070BD4FF48071864807F0EBFC044611
:1005200018B9FFF72DFF204602E0FFF721FF012059
:1005300029687E4A0129804B08D003D302297F4EC7
:1005400015D02BE001211160186070BD1A6890422F
:1005500000F08781002818600CBF02220322784B2C
:100560002A60FF221A60754B00221A6070BD19685C
:10057000884202D1336801330EE0186033680321EA
:10058000782B116003D96E4B00221A6003E04A2BCE
:1005900001D800232B600023336070BD19688842A6
:1005A000E8D018603368022111609A1F122A644C47
:1005B0000BD9052B94BF6348634804F02BF96348BB
:1005C00004F028F900232B6000E10F2B236840F290
:1005D000E980113B292B00F2F980DFE813F02A00B3
:1005E000F700F700F7002E00320036003F0043000E
:1005F00047004B004F0056005A006000640068003E
:100600006C007000770079007B007D007F00810026
:1006100083008500870089008B008D008F0091008A
:10062000930097009B009F00A300CF00D300D7004A
:10063000DD00474B01221A60C8E0464A13680133C7
:1006400006E0444A1368023302E0424A1368043366
:100650001360414A136801331360B7E03D4A1368E1
:100660000833F5E73B4A13680A33F1E7394A136860
:100670001433EDE7374A13682833E9E7364B1B6834
:10068000DA0700F1A380354897E7354A136801334C
:1006900002E0334A136802331360324ADAE7304A21
:1006A00013680433F8E72E4A13680833F4E72C4A3A
:1006B00013680A33F0E72A4A13681433ECE7294B2E
:1006C0001B68DB0700F18280274876E7274A1AE09B
:1006D000264A1CE0254A1EE0244A20E0234A22E064
:1006E000224A4CE0224A0EE0214A10E0204A12E061
:1006F000204A08E01F4A0AE01E4A0CE01D4A0EE0AC
:100700001C4A10E01C4A1368013342E01A4A13687D
:1007100002333EE0184A136804333AE0164A13687D
:10072000083336E0144A13680A3332E02000002010
:10073000B8030020000C0140C0030020AC030020DF
:100740001C00002003A4000820A40008E7B1000852
:10075000CC030020B4030020B00300203EA4000816
:10076000D8030020D00300205FA40008A8030020C5
:10077000BC030020E0030020A4030020394A1368D2
:10078000143306E0374A1368283302E0354A136809
:1007900050331360344A5DE7334B1B68D80715D4D8
:1007A00032480AE7232B08D03A2B0BD01C2B0DD153
:1007B0002F4B1B68D90709D565E72E4B1B68DA0755
:1007C00004D581E7284B1B68DB07E9D422680F2A90
:1007D00009D1294B1A68002A40D0284A012111600A
:1007E00000221A603AE0102A19D1244900230B6034
:1007F00021490B601E490B601E490B601A490B60B2
:100800001F490B601F490B601F490B601F490B609C
:100810001F490B601F490B6012490B6002E0FF2A61
:100820003FF4B9AE01323B2A226014D1164A1A4B6A
:1008300011681868134C8842184807D10168256868
:100840000131A94202BF0C4901250D6012681A60EE
:10085000236803609FE63FF69CAE9CE6102323606E
:1008600099E670BDA4030020D403002080A40008F2
:10087000B0030020D0030020E4030020C8030020C0
:10088000CC030020B4030020D8030020BC030020C8
:10089000A8030020E0030020C4030020DC030020A4
:1008A000034B1A6812B11A68013A1A60704700BF08
:1008B0001C120020054B1A68054B012A18BFB0FB1B
:1008C000F2F018601A68002AFCD170472800002056
:1008D0001C120020044B1B685843044B18601A6814
:1008E000002AFCD1704700BF240000201C12002009
:1008F000014608B529B14FF47A70FFF7EBFF0139D3
:10090000F8E708BD002808BF64204FF47A73B3FBF2
:10091000F0F30D4A13600D4BB3FBF0F20C4B1B6868
:10092000B3FBF2F3B3F1807F0AD20A4A013B536072
:10093000094BF02183F823100023936007231360F1
:10094000064B1860704700BF2400002040420F0093
:10095000C002002010E000E000ED00E028000020D0
:10096000074A02F16E0112F8013F98074CBF43F0AD
:10097000040323F004038A421370F4D1704700BFCC
:10098000330400200B4BDA681A6193F8482083F88F
:100990004B2093F8492083F84C2093F84A2083F8A1
:1009A0004D20054A054B117819705178927859708D
:1009B0009A707047300000202C00002014020020A4
:1009C00037B51D4B002419601C4B8DF8044018608E
:1009D0008DF805408DF8064028B3194A194B107858
:1009E00033F810008DF800005078927833F810003A
:1009F00033F812308DF801008DF802300523B1FB79
:100A0000F3F303EB8303CD1AA5428CBF694601A91A
:100A10002046013406F064FF042CF5D1042006F0D2
:100A2000F7FE03B030BD0446204601A9013406F0AC
:100A300057FF042CF8D1F1E7B0050020E8030020AF
:100A40002C000020D4A40008034BDB6A13B1AE20B5
:100A500006F0DEBE704700BF3000002070B50646CD
:100A60000D46722420463146013406F039FFAE2C83
:100A7000F8D11DB1BDE87040FFF7E6BF70BD0000C2
:100A800007B50C4A0C4B117833F811108DF804108F
:100A90005178927833F8111033F812308DF8051030
:100AA000014601A88DF80630FFF7D8FF03B05DF8C6
:100AB00004FB00BF14020020D4A4000807B50023E3
:100AC000014601A88DF804308DF805308DF8063008
:100AD000FFF7C4FF03B05DF804FB00001FB5084B2F
:100AE000002253F8041F0DF802100132102AF8D129
:100AF000694640F2EF1002F03FFD05B05DF804FBDF
:100B0000CC01002007B50A4B01A993F84820A42086
:100B10008DF8042093F8492093F84A308DF8052089
:100B200003228DF8063002F027FD03B05DF804FBC8
:100B30003000002007B5064B02A91B68012201F80E
:100B4000013DA72002F018FD03B05DF804FB00BFD3
:100B50003000002007B5064B02A99B69012201F86D
:100B6000013DBC2002F008FD03B05DF804FB00BFAE
:100B70003000002007B5064B02A9DB69012201F80D
:100B8000013DA82002F0F8FC03B05DF804FB00BFB3
:100B90003000002007B5064B02A99B68012201F82E
:100BA000013DA92002F0E8FC03B05DF804FB00BFA2
:100BB0003000002007B5064B02A9DB68012201F8CE
:100BC000013DBD2002F0D8FC03B05DF804FB00BF7E
:100BD0003000002007B5064B02A95B69012201F82D
:100BE000013DBE2002F0C8FC03B05DF804FB00BF6D
:100BF0003000002007B50A4B01A993F84B20D720FD
:100C00008DF8042093F84C2093F84D308DF8052092
:100C100003228DF8063002F0AFFC03B05DF804FB50
:100C20003000002007B5064B02A91B69012201F81C
:100C3000013DDA2002F0A0FC03B05DF804FB00BF28
:100C40003000002007B5064B02A95B68012201F8BD
:100C5000013DDB2002F090FC03B05DF804FB00BF17
:100C60003000002007B5064B02A95B6C012201F899
:100C7000013DDC2002F080FC03B05DF804FB00BF06
:100C80003000002007B5064B02A91B6C012201F8B9
:100C9000013DDD2002F070FC03B05DF804FB00BFF5
:100CA000300000200B2807B50ED80D4A142303FB93
:100CB0000022936D126E03F00F0392078DF8073038
:100CC00005D543F0100300E0FF238DF80730012223
:100CD0000DF10701E53002F04FFC03B05DF804FBB5
:100CE0003000002007B5012897BF0B4BFF2303EB13
:100CF0000013D3F844314FF0010298BF03F00F0303
:100D00000DF1070100F225108DF8073002F034FCD8
:100D100003B05DF804FB00BF30000020032807B5D6
:100D200011D80F4A02EB001302EB0012D3F8643122
:100D3000D2F86C2103F00F0392078DF8073005D528
:100D400043F0200300E0FF238DF8073001220DF16E
:100D5000070100F2351002F00FFC03B05DF804FB50
:100D60003000002007B5074B02A9D3F8E03101227B
:100D700001F8013D40F27F2002F0FEFB03B05DF878
:100D800004FB00BF3000002070B5234B8CB01C6A00
:100D90001E4664B300242346142202FB0361096E3D
:100DA000890742BF0CA901EB840141F8303C03F1F3
:100DB000010348BF01340C2BEFD1184D0CB92C6046
:100DC0000BE007F0E9FEB0FBF4F303FB14000CABFF
:100DD00003EB800050F8303C2B602A68142303FB9F
:100DE00002635B6D98470E4B00221A6011E00B4ABC
:100DF000142512680A4805FB023301689A6D013117
:100E00009142016005D35B6D04600CB0BDE8704099
:100E100018470CB070BD00BF30000020B4050020A2
:100E2000F80500202DE9F74F00930B0622D5DC29A9
:100E30001BD007D8C4291CD0D62912D0B02916D16E
:100E4000012117E0E4290AD003D8DF290FD10821B6
:100E500010E0F62907D0FC2909D107210AE0052175
:100E600008E0032106E0062104E0042102E020213D
:100E700000E00221284C00F10B062644C90000279F
:100E800001944FF001094FF00B0B3546234B02F153
:100E9000010CC2F1040E002403EB070ABCF1050F9C
:100EA00022D804EB0008B8F10A0F16D81AF801800E
:100EB000009B48FA0EF84BB118F0010F0DD095F8D1
:100EC000008048F0020885F8008006E018F0010F65
:100ED00016BF042385F800902B7001340CF1010C2F
:100EE00001350EF1FF3ED9E7009B3BB10137082FDA
:100EF00006F10B06C9D103B0BDE8F08F0BFB07FE6E
:100F000004440A2CF2D8019B04EB0E051D4485F81D
:100F10000B900134F5E700BF340400205BA8000803
:100F2000722006F075BC70476D2838B5154610D88C
:100F30000B23B0FBF3F4E20742BF6343C0EB430073
:100F40000A30043006F0CCFC1DB1BDE83840FFF794
:100F5000E7BF38BD73B50546144A154B1178002418
:100F600033F81110134E8DF800105178927833F841
:100F7000111033F812308DF801108DF802308DF811
:100F800004408DF805408DF80640A25D20462A40B9
:100F90001ABF0022694601A90134FFF7C5FF6E2C74
:100FA000F3D1FFF7BDFF02B070BD00BF2C000020E1
:100FB000D4A400083404002038B5184C236A23B1A7
:100FC000174A0023236263621360636A23BB144DD4
:100FD0002B6801332B6007F0DFFD124B00F0070098
:100FE00003F16E0101281A7805DD12F0030F02D01B
:100FF00042F0040201E022F004021A7001338B4235
:10100000F0D12B68202B03BF012363620220042050
:10101000BDE83840FFF79EBF38BD00BF300000205C
:1010200030040020340400202DE9F047384D2B6AAD
:1010300023B1384A00232B626B6213606C6A002C68
:1010400064D1344E3368A3BBDFF8CCC01C461A46CB
:10105000E2464FF00B0909FB02FE0CEB0E00804646
:101060000B277B1EC15C11F0010F14D00A2B02D09C
:10107000C45DE4070ED421F0010108F803103BB170
:10108000013B03EB0E0151444978C90702D5F6E74D
:10109000012403E001240BB11F46E2E701320A2AD2
:1010A000D9D10120FFF756FF01230CB9336000E0CE
:1010B0001C463368012B29D1174F00214FF00B0E2E
:1010C0000EFB017630460023C25C02F0060CBCF138
:1010D000020F0FD113B112F0040F0BD142F0040232
:1010E000C2540A2B05D05A1CB45CA40701D5134680
:1010F000F7E7012401330B2BE6D101310A29DFD1B7
:101100000420FFF727FF0CB901236B62BDE8F087CD
:1011100030000020E4040020340400202DE9F04FCA
:10112000764B85B01A6A3AB1002275491A625A6242
:1011300001220A6073490A605B6A002B40F0DA8082
:101140006F4B1D68184655B36F4D0A210B264A1E7A
:1011500006FB02570023FC5C04F0030EBEF1010FF6
:1011600010D169480B2505FB020024F00104092A6F
:10117000C4540ED0644A05FB0121CA5C42F001024E
:10118000CA5406E001330B2BE5D11146002ADED10B
:101190000260052005B0BDE8F04FFFF7DBBE594BFC
:1011A0001A680393002A00F09D80584E584833680F
:1011B0005849594FE3B10268DFF84CE10B2303FBB8
:1011C00002EC096801321CF8014003FB02E324F041
:1011D00004040CF801400260585C40F004045C54C4
:1011E0003C68A242D5D140F0050058543560D0E7A4
:1011F0000268D7F800E018460F689B461C469C46DC
:1012000019460292454A4FF00A080192A2F16E096E
:1012100008F1FF350022002945D1019EA6F10B0AF5
:101220001AF802A00AF00306022E38D12DB32C467C
:101230000AF00101013C81B1019B01999B5C0120F5
:1012400043F004038B54CDF808801746AE4603469E
:10125000834604468446014621E0002CEAD1C3B906
:1012600012F80910029341F00401012302F8091059
:101270001746AE4618469B460EE012F809100124A8
:1012800041F0050102F809101746AE46A446214672
:1012900005E01746AE4601231C469C46194601321E
:1012A0000B2AB8D100E00121019AA8460B3A01921D
:1012B000002DADD1BCF1000F02D0174AC2F800E0FA
:1012C0000CB1144A1760BBF1000F02D0104A029C07
:1012D000146008B10D4A136000297FF45AAF039BD4
:1012E000196056E7FFF73CFB0420FFF733FE034B82
:1012F00001225A6205B0BDE8F08F00BF3000002027
:10130000CC050020B0040020340400200C0600208E
:10131000F405002064050020F0050020A204002050
:101320002DE9F041534B1A6A22B1534900221A6247
:101330005A620A605B6A002B40F09A804E4C236828
:10134000042B3ED84D4A6FF00A000C21584301FB94
:101350000321C3F10B05801A4718BD42474E05D93A
:101360000E7846F0040601F8016BF5E70A2101FB4F
:101370000361581CC3F10907B84201F10B010DD2FA
:1013800011F813E001304EF0040E01F813E091F86B
:101390000AE04EF0040E81F80AE0EDE70B2101FBB4
:1013A00007316FF00A000A4400FB07F1891B10782F
:1013B00040F0040002F8010B88188542F7D89BB171
:1013C0001AE0052B4CD117E00B2202FB0102BB18DF
:1013D0006FF00A024A43921B197821F0040103F8C6
:1013E000011BD1188D42F7D80420FFF7B3FD236805
:1013F00001332360BDE8F081581E0B2141436FF09B
:101400000A0E0EFB00FE1D4F42183A44C0F10B05B8
:10141000C7EB0E0E0EEB020C6545184E05D916787B
:1014200026F0040602F8016BF4E70B310144721850
:10143000C3F1000CC0F109018B4202F10B02C3D2CF
:1014400012F80BECC0EB02082EF0040E02F80BECC5
:1014500018F80CE001332EF0040E08F80CE0EBE76E
:10146000FFF77EFA0420FFF775FD024B01225A6256
:10147000BDE8F08130000020D005002034040020B9
:1014800038B5204A136A33B11F4900230B601F4946
:10149000136253620B60536A002B31D11A4C2368DC
:1014A0006BB91B4B03F16E0113F8012F22F00402FC
:1014B0008B421A70F8D10420FFF74CFD1CE0134852
:1014C000016801310160C9071AD5013B11489BB27F
:1014D0006D2B0FD8C15C5D1C11F0020F08D00D4AB6
:1014E00041F004010420D154FFF734FD256003E0EE
:1014F000ABB2EDE70123536223680133236038BDAB
:1015000038BD00BF30000020A80400207005002076
:1015100033040020340400202DE9F04F784B85B0CF
:101520001A6A22B1774900221A625A620A605B6A1B
:10153000002B40F0E280734A17681146042F00F236
:10154000D980714D0022EC18A05CDFF8BC8120F03E
:101550000400A05401320B2AF6D10B336E2BF1D1CB
:1015600007F1010BC1F800B0CBF105060022002302
:1015700008EB0200C15C21F00801C15401330B2BC0
:10158000F8D10B326E2AF2D10020C6F1000A55467E
:1015900003FB0082C6EB000CBCF1050F06EB000E4E
:1015A00038BF4FF0050CBEF1040F01924FF000015F
:1015B00028BF4FF0040E019A525C940720D50428EE
:1015C00009D80429744604D87218042A28BF0422B2
:1015D0000EE0042D09E0042905D87218042A28BF5A
:1015E0000422644604E06446042D8CBF2A4605228A
:1015F00003FB048414F8029049F0080904F80290EF
:1016000001310B2905F10105D5D101300A28BED1E0
:1016100000225D4610460C237B43029316237B4336
:1016200039494FEA470E03935C46029B8F18C3EB80
:101630000209039B0EEB090803EB080CCEEB0C032D
:1016400001930023FE5CF6073CD504281DD8042B2B
:101650000DD8834536D89B4534D803EB09060E4494
:1016600016F80CAC4AF0040A06F80CAC2AE08345E4
:1016700028D80A2C26D803EB08060E4416F80AAC24
:101680004AF0040A06F80AAC1CE0042B0DD8092D18
:1016900018D89B4516D8019E9E190E4496F80AA0AC
:1016A0004AF0040A86F80AA00CE0092D0AD80A2C90
:1016B00008D80CEB03060E4496F80CA04AF0040A76
:1016C00086F80CA0FE5C013416F0080F1CBF46F033
:1016D0000406FE5401330B2BB4D10B326E2A00F1F9
:1016E000010005F101059FD1042005B0BDE8F04FD0
:1016F000FFF730BC024B01225A6205B0BDE8F08F03
:1017000030000020C404002034040020F8B5774CD9
:10171000774D236A5BB107F03FFA764B0340002B0D
:10172000BEBF03F1FF3363F0030301332B602B686B
:10173000032B00F2DA80DFE803F0023670A4236A9C
:101740006A4A23B10023136253626B4A1360626AD0
:10175000002A40F0CA80684B18680A2854D8674E9F
:10176000471CB6461F60B3180021151A6C188F422B
:10177000744404D814F8014C14F0010F02E0A47A68
:1017800014F0020F1C7801F1010114BF44F00404AD
:1017900024F004040B291C7003F10103E6D10B3281
:1017A0006E2AE0D12BE0236A504A23B10023136252
:1017B0005362534A1360626A002A40F09680504B8D
:1017C00018680A2820D8461C4C4F1E600C30BC18E4
:1017D000234631460A291AD8655C15F0010F1D7899
:1017E00001F1010114BF45F0040525F00405814213
:1017F0001D7003F10103EDD10B326E2AE7D1BDE874
:10180000F8400420FFF7A6BB01236362F8BD65180A
:1018100015F80B5C15F0020FE1E7236A334A23B198
:10182000002313625362374A1360626A002A5CD154
:10183000344B1D686D2DE7D805F10B062F481E604F
:1018400002F10B04831807199642A3EB050104D893
:1018500011F80B1C11F0010F03E091F8631011F067
:10186000020F197803F1010314BF41F0040121F0C4
:10187000040103F8011CBB42E6D16E2C2246DFD1E5
:10188000BDE7236A194A23B10023136253621E4A3B
:101890001360636A4BBB1C4B1D686D2DB4D805F1FA
:1018A0000B02164E1A600B24A4F10B0333443019BB
:1018B00061196D2903EB050203D8D27A12F0010FEA
:1018C00003E012F8632C12F0020F1A7803F10103FF
:1018D00014BF42F0040222F0040203F8012C9842E3
:1018E000E7D10B34792CDFD189E7F8BD3000002037
:1018F000D804002003000080BC0500203404002030
:10190000AC040020D8050020D0040020F8B5194D03
:10191000194F2E683C680023224631781846FFF79D
:1019200081FAC4F1060416F8011F91B10A2C06D8F9
:10193000002320461A46FFF775FA0634F3E7042021
:10194000FFF708FB3B680C4A0133062B0BD01360F2
:10195000F8BD0A2CF3D8002320461A462021FFF7B1
:1019600061FA0634F5E7002313602B6801332B601E
:10197000F8BD00BF20020020EC05002030B5694909
:1019800085B00B6A3BB300230B624B62664B14229B
:101990001C786648B4FBF2F20AB904B10122026075
:1019A00058781422B0FBF2F2614D0AB900B101225D
:1019B0002A609A781423B2FBF3F35E4D0BB902B19F
:1019C00001232B605C4B00251D705D709D705B4B8F
:1019D0001C7058709A704C6A002C40F0A080534BD9
:1019E0001A68BAB1554803789A4202D89B1A037014
:1019F00001E00BB1047001234F484B4C057824786B
:101A00002A44A24201D8027002E0A54203D0047029
:101A1000012300E01346464A1268BAB1474C607889
:101A2000824202D8801A607002E010B10023637015
:101A3000012341483C4C457864782A44A24201D8AD
:101A4000427002E0A54201D044700123394A126875
:101A5000BAB13A4CA078824202D8801AA07002E053
:101A600010B10023A370012333482F4C8578A4784C
:101A70002A44A24201D8827007E0A54201D08470B6
:101A800003E013B901234B6249E0274A2C4B11783C
:101A90002C4D33F8111000248DF8041051789278F1
:101AA00033F8111033F812208DF805108DF8062048
:101AB000214A117833F811108DF808105178927876
:101AC00033F8111033F812208DF809108DF80A2020
:101AD0001A4A117833F811108DF80C105178927859
:101AE00033F8111033F812308DF80D108DF80E30D8
:101AF000635D022B02D1002202A908E0012B02D172
:101B0000002203A903E0032B04D1002201A92046EF
:101B1000FFF70AFA01346E2CEAD1FFF701FA05B09B
:101B200030BD00BF300000202C0000206C050020DC
:101B3000E004002014060020B4040020B7040020B4
:101B4000D4A400083404002073B5274B06461A6855
:101B50000AB901261E60254A254B1178002433F866
:101B60001110244D8DF800105178927833F811102F
:101B700033F812308DF801108DF802308DF80440E2
:101B80008DF805408DF8064015F8013F03F002037B
:101B900003F0FF0243B1002269462046FFF7C4F973
:101BA0002B7843F0010306E001A92046FFF7BCF9BA
:101BB0002B7823F0010301346E2C2B70E4D10E4BF3
:101BC0000E4C19680E4B1868FEF7FAFE2EB16368CA
:101BD0001BB90120FEF754FF01E0FFF7A1F9012333
:101BE000636202B070BD00BFDC0400202C00002046
:101BF000D4A4000833040020B005002030000020E9
:101C0000E803002010B5054C236A1BB100202062B8
:101C1000FFF79AFF0123636210BD00BF3000002070
:101C2000084B10B503F16E00012413F8011F01F0F9
:101C30000201002901F0FF0218BF224683421A70F8
:101C4000F3D110BD330400200E2A10B50C7804D94E
:101C500004704B7843708B7826E01BB1134B6832CD
:101C600053F8222054430F23B4FBF3F3DBB2037089
:101C70000C7814B10BB9012303704B780F24534334
:101C8000B3FBF4F3DBB243704C7814B10BB901230E
:101C900043708B785A430F23B2FBF3F2D2B28270B7
:101CA0008B7813B10AB90123837010BD3000002076
:101CB0002DE9F04F694D85B02B6A002B56D0684B4B
:101CC00000241C603F238DF800308DF801308DF822
:101CD000053010238DF80630EA680123694602A812
:101CE0002C626C628DF802408DF80440FFF7ACFF67
:101CF0000123EA6801A903A8FFF7A6FF594B9DF845
:101D00000810594A33F81110584F11709DF80910F6
:101D10000A2633F8111051709DF80A1033F811108B
:101D200091709DF80C10524A33F8111011709DF803
:101D30000D1033F8111051709DF80E1033F811305A
:101D40009370E30706D506F027FF90FBF6F303FB3D
:101D5000160006E006F020FF90FBF6F303FB1600EA
:101D6000053047F8240001340B2CEAD16C6A002CB2
:101D700070D13B4B1A6898461D2A63D83C4EDFF859
:101D8000F49033788DF80C3073788DF80D30B3788B
:101D90008DF80E3059F8043F0F2B0FD8D9F80030CA
:101DA000013401330B2CC9F80030F3D1FFF7B8F838
:101DB000D8F800300133C8F800304BE0A3F10F052C
:101DC000012D07D10B200022274900FB0540FFF71A
:101DD000ABF80DE0113B092B08D8A4F116000B233A
:101DE0000022234903FB0500FFF79EF8092DE9D9DE
:101DF0004FF0010A4FF00B0B6F1E092F0FD9AF1ECA
:101E0000033D082D18D873780022B3FBFAF303A919
:101E10000BFB07408DF80D30FFF786F80CE0737868
:101E20000022B3FBFAF303A90BFB07408DF80D303A
:101E3000FFF77AF8002FE2D10AF1010A002FADD0A6
:101E40003D46D9E7FEF78CFD0420FFF783F8034BEE
:101E500001225A6205B0BDE8F08F00BF30000020BB
:101E6000E4050020D4A40008E80500207C0500203B
:101E7000DC050020780500202DE9F74F8F48036A24
:101E800063B18F4A002313608E4A036213608E4A47
:101E9000436213608D4A13608D4A1360436A874E14
:101EA000002B40F00881864C864D2368002B51D1D1
:101EB00096F848201F2A05D83F228DF800208DF87B
:101EC000013008E096F849201F2A07D83F228DF8F4
:101ED00000308DF801208DF802300DE096F84A2090
:101EE0008DF800301F2A4FF03F0294BF8DF801306B
:101EF0008DF801208DF80220C2680123694601A8EF
:101F0000FFF7A2FE734B9DF80420734933F81220AB
:101F10006D4E0A709DF80520286833F812200B27B3
:101F20004A709DF8062033F8123000228B706B4BFC
:101F30001A705A709A70336807FB0030FEF7F4FF8E
:101F400023682968664AD1543168664AD1540133FE
:101F50002360A9E02A680F2A07D9FEF701FD0420B3
:101F6000FEF7F8FF01237362A5E0584B564E19683F
:101F70009E468A42DFF8588102F0010942D1316859
:101F8000D8F8003099423DD1B9F1000F02D031B1FB
:101F9000013902E0092902D80131924601E002F13B
:101FA000010A5746504B4FF00B0C0CFB0A3C092F13
:101FB00025D8BA4507F0010B04D0BBF1000F03D1BF
:101FC0005B4619E00B4600E00A23BBF1000F13D07B
:101FD0000133002B6BD0013B1CF803B01BF0010F49
:101FE000F7D0CEF80070C8F800300BE01CF803B052
:101FF0001BF0010FF5D101330A2BF7D957E010235D
:10200000CEF800303368D8F80010B9F1000F03D0D3
:102010008B4207D9013B02E08B4203D201332A4AAB
:10202000136007E0DEF800309A4235BF0132012329
:102030002A6043622B68092B07D830680B270022DF
:10204000254907FB0300FEF76FFF2368DFF8908048
:10205000062B244F1DD198F80030092B08D838786A
:102060004FF00B0E00221D490EFB0300FEF75CFF34
:102070000023013318F8031008EB030202F8011CD7
:10208000F95CFA18052B02F8011CF2D12368013B18
:10209000236023682A68052B08F803203268FA5465
:1020A0009EBF074A01331360FEF73AFF03E0013792
:1020B0000CF10B0C7BE703B0BDE8F08F3000002083
:1020C000BC040020D40400201806002010060020C4
:1020D000B8050020D4A40008680500207805002079
:1020E000FC050020A80500203404002037B5104D61
:1020F000104C01232A6905F14B012046FFF7A4FD8E
:10210000EB6A9BB10C4B2278012133F8122001A815
:102110008DF80420627833F812208DF80520A2781B
:1021200033F812308DF80630FEF798FC03B030BD5E
:102130003000002014020020D4A400080D4B5A687F
:10214000032A16D8DFE802F00208050BD86AFEF76A
:1021500097BC094B01221A600020FEF7AFBC3F225A
:1021600083F84B20002283F84C2083F84D20FFF7A2
:10217000BDBF7047300000200806002010B50C4C91
:102180000123E26804F148010A48FFF75DFD636836
:10219000032B04D0A3699B0701D5FEF7F3FBA36AC9
:1021A00023B1BDE810400120FFF7CEBC10BD00BF39
:1021B000300000202C000020074B9A68012A09D12A
:1021C0003F2283F84820002283F8492083F84A20E0
:1021D000FFF7D4BF704700BF3000002038B5054678
:1021E000064C28B10123E362BDE83840FEF72CBC61
:1021F0000120FEF763FCE56238BD00BF300000201F
:102200002DE9F74F044688469246002A00F0B68032
:102210000020FFF799FC1AF0080F5A4E0AD003F07D
:10222000A9FFC820FEF756FB73684BB90120FEF7E3
:1022300027FC05E01AF0100F02D00120FEF73EFC4B
:102240004146B06AFEF7BCFB1AF0040FDFF834B168
:1022500000F094800525B8FBF5F5DBF800904822E6
:1022600002FB09F1062202FB0512474B00219F5C8D
:1022700046487622019306F0DCFBFFF7D1FCDBF841
:102280002820019B002A74D0DBF8182012F0010FDF
:102290003E4A07D1B8F1040F04D9A8F11E08B8F1DD
:1022A000040F13D8482101FB09F1062000FB05119A
:1022B00019444978364801F0030100EB410E10F84B
:1022C0001100012111549EF8010011544FF0060E27
:1022D0000EFB05FE482101FB09EE4FF0010C002129
:1022E00001EB0E001844807820B10131042902F876
:1022F00000C0F5D10B2C00D90C3C482101FB09F999
:10230000062101FB05951D446B7801205B0748BF42
:1023100001340B2C88BF0C3C242304EB440403FB46
:1023200007441C4B1C44631E023413F8011F11B1F7
:10233000A3425054F9D11849DFF860E000200B2780
:10234000135C2BB90130762801F10301F8D113E0B9
:1023500011F8013C0D784C7807FB0353013B7344A3
:1023600014F1FF34EED313F8015F45F002051D7040
:10237000F6E71AF0100F01D00123336203B0BDE875
:10238000F08F00BF300000207FAC0008E804002080
:1023900079AC00087CB000081BAF000834040020B2
:1023A000F0B5D14B0546186891B00024002800F024
:1023B000B1813F238DF81C303C2303268DF80B3070
:1023C00016238DF80C3032460F2306A9A4208DF871
:1023D00011308DF807408DF81D408DF81E408DF8A6
:1023E00008408DF80D408DF80E408DF80F608DF887
:1023F000136001F0A9F801220DF10901A72001F0F5
:10240000A3F801220DF10D01A82001F09DF8012291
:1024100004A9BD2001F098F801220DF11201BE209F
:1024200001F092F8B5F5843FC0F09F8001220DF1D4
:102430000E01A92001F088F8AC4B9D4240F2958036
:1024400001220DF10F01BC2001F07EF8324607A9F0
:10245000D72001F079F801220DF11101DA2001F005
:1024600073F801220DF10A01DB2001F06DF8B5F5DA
:10247000003F7AD301220DF10B01DC2001F064F85A
:10248000012203A9DD2001F05FF8994B9D426CD930
:1024900009AF0C223946E52001F056F808AE0222B9
:1024A00005A940F2251001F04FF83146042240F210
:1024B000351001F049F88F4B19463A5DFF2A0BD0D1
:1024C00012F0100F02F00F001A6E986514BF42F060
:1024D000020222F002021A6601340C2C03F11403EA
:1024E000EBD19DF814300020FF2B1CBF03F00F032D
:1024F000C1F844319DF81530D1F87C21FF2B1CBF69
:1025000003F00F03C1F8543103467B4FF45CFF2CFA
:1025100010D001EB031E04F00F0CBD42CEF864C1D5
:1025200008D9012B06D1A40601D40223EEE71846F0
:1025300042F002020133042BE8D108B1C1F87C213A
:102540006E4B9D4211D901220DF1070140F2451059
:1025500000F0FAFF012202A94FF4A37000F0F4FF8B
:10256000674B9D4201D1022226E0B5F5013F00F004
:10257000CF8030D90CAC1022214640F2EF1000F091
:10258000E3FF604A00230F20E15C01330F298CBF79
:10259000106011600F2B02F10402F5D1554AC2F808
:1025A000DC31554B9D4206D901220DF1130140F259
:1025B0007F2000F0C9FF0522534940F2971000F038
:1025C000C3FF524B00215A1D13F8010F3C2888BF4E
:1025D00019709A42F8D19DF80930072B02D90023CF
:1025E0008DF809309DF80A30424C032B84BF00233C
:1025F0008DF80A309DF80D300B2B84BF00238DF829
:102600000D309DF80E30012B84BF00238DF80E3065
:102610009DF810300F2B84BF0F238DF810309DF8DC
:1026200011300F2B84BF0F238DF811309DF812301D
:10263000012B1CBF00238DF812309DF80B303C2B72
:1026400084BF3C238DF80B309DF80C303B2B84BFAE
:1026500016238DF80C309DF8093023609DF80A3060
:1026600063609DF80F30A3619DF80D30E3619DF824
:102670000E30A3609DF8183084F848309DF819306A
:1026800084F849309DF81A3084F84A309DF81C309F
:10269000A56A84F84B309DF81D3084F84C309DF8C5
:1026A0001E3084F84D309DF81030E3609DF81130F5
:1026B00023619DF8123063619DF80B3063649DF8CF
:1026C0000C3023640023A362FFF710FDFFF756FDD3
:1026D0009DF81330A562C4F8E031FFF76DFDFFF7F8
:1026E0002DFD012016E000BF38060020FF08010084
:1026F000FF00020030000020FF050200FF01020081
:1027000000030200D00100206400002063000020CC
:10271000042251E711B0F0BD0F2928BF0F2110B5D9
:102720000C46044B683043F82010FEF7D7F92046DA
:1027300010BD00BF3000002010B51E4B1868B8B3A4
:10274000FEF7E0F9FEF7F6F9FEF704FAFEF712FAE3
:10275000FEF720FAFEF72EFAFEF73CFAFEF74AFAE9
:10276000FEF760FAFEF76EFAFEF77CFAFEF78AFAD9
:102770004022114940F2971000F0FEFE002420464E
:102780000134FEF78FFA402CF9D1002420460134A1
:10279000FEF7A8FA102CF9D1002420460134FEF7E8
:1027A000BDFA102CF9D1FEF799F9FEF7DBFA0120FA
:1027B00010BD00BF380600206400002010B5044C96
:1027C000C4F8E001FEF7CEFAD4F8E00110BD00BF76
:1027D0003000002038B50A4C05466368032B06D04C
:1027E000820704D5A3699B0701D4FEF7CBF8FFF756
:1027F000A5FC0123A5612362FEF7ACF9A06938BDF1
:1028000030000020032838B50D46074C0AD863680D
:10281000984207D06060FFF791FC0DB104F0DCFB3B
:10282000FEF710FA606838BD3000002010B53B2874
:10283000044C8ABF3C2360646364FEF713FA606C47
:1028400010BD00BF3000002010B53A28044C8ABFEC
:10285000002320642364FEF715FA206C10BD00BF2E
:1028600030000020072810B5054C07D80123206050
:10287000236209B104F090FBFEF75CF9206810BDFB
:102880003000002010B5084C2368062B94BF01339C
:10289000002323600123236208B104F07DFBFEF7CF
:1028A00049F9206810BD00BF3000002010B5084C69
:1028B00023680BB9072300E0013B23600123236257
:1028C00008B104F069FBFEF735F9206810BD00BFC0
:1028D000300000200B2810B5044C05D8E06109B188
:1028E00004F072FBFEF746F9E06910BD30000020ED
:1028F00010B5074CE3690A2B94BF01330023E36151
:1029000008B104F061FBFEF735F9E06910BD00BFC6
:102910003000002010B5074CE3690BB90B2300E031
:10292000013BE36108B104F04FFBFEF723F9E069D6
:1029300010BD00BF30000020012838B50D46074CFF
:102940000AD8A368984207D0A060FFF735FC0DB104
:1029500004F052FBFEF71EF9A06838BD30000020DD
:10296000F0B5664D85B06B680446012B1AD1002086
:10297000FEF7A4F86B6C3B2B03D92B6C1C443C2357
:102980002EE01D2B04D92B6C03EB54041E2327E0EF
:10299000132B40F2B1800323B4FBF3F42B6C1C44E3
:1029A00014231DE0022B40F0A78030B9544B1A6865
:1029B0000AB1186001E001221A600020FEF77EF8DB
:1029C0006B6C3B2B5ED81D2B02D964081E265AE087
:1029D000132B40F291800323B4FBF3F4142652E04E
:1029E0009C4200D3E41AD5F87C21464E12F0020F27
:1029F00030D03C2B2ED1444B02A91A889B78ADF8DD
:102A000008203E4A8DF80A301269012303A8FFF717
:102A10001BF99DF80C30002736F813308DF8043080
:102A20009DF80D3036F813308DF805309DF80E30D6
:102A300036F813308DF80630286C38443B2802D91C
:102A40003C383B2803D801A9723004F049FF053710
:102A50003C2FF1D12D4B3B2C1A7836F812208DF8F3
:102A60000C205A789B7836F8122036F813308DF8FF
:102A70000D208DF80E3025D803A904F1720004F062
:102A80002FFF1FE03C26214A1E4B117833F811100E
:102A90008DF80C105178927833F8111033F8123009
:102AA0008DF80D108DF80E30154B1B68E3B1002723
:102AB000286C3844B0420AD3801B3B2807D9013721
:102AC000A742F5D9EB6ABBB1FDF7BEFF14E003A93D
:102AD000723004F005FFF2E7286C2044B04206D3C0
:102AE000801B3B2803D90134B442F5D3EAE703A99C
:102AF000723004F0F5FEF6E705B0F0BD30000020BE
:102B000008060020D4A40008A1A400081402002094
:102B1000F8B5134B0F469A6A1E46FAB1114D2023A1
:102B20003E220146A81C2B706B700F4C06F0D6F8A5
:102B30000E4B00221A602560FFF772F807B9F8BD46
:102B40004FF47A7523681B7843B1FEF7DFFED6F8A1
:102B5000E00168438009FDF7BDFEF3E7F8BD00BF63
:102B600030000020EC03002020020020EC050020B3
:102B70002DE9F04F9F4B87B01B689F4C1B786BB1C2
:102B80009E4AD4F8E011136801338B421360C0F001
:102B9000FD8100231360FEF7B9FEF7E1256BFF2DE1
:102BA0005FD0A26A002A00F0F1818DF814308DF810
:102BB00015308DF81630924BDFF878821A689946F6
:102BC000FF2A27D18F4E1D602D017319D8688E4CB6
:102BD00008B106F066F82060002472197359264681
:102BE000C3F10A0389495B080B605368884AC3F143
:102BF0000B035B08874DC8F80040136066552046FC
:102C0000002205A90134FEF78FF96E2CF6D1FEF7EC
:102C100087F9BBE1D8F800300133DA07C8F8003093
:102C200014D5E2687F2B02F1680288BFC3F1FF036D
:102C300054F822705B089F4280F01E81724B1B6823
:102C4000002B40F01A8101E0FEF76AF9D8F8003055
:102C5000B3F5807F40F09A81FF23C9F800302363E9
:102C600094E1E3690B2B21D8A26A1AB9226A0AB946
:102C7000626AFAB9226A60491AB1142202FB03138C
:102C800012E04D6AB5B9042B02D1D1F8A4300CE0A2
:102C9000142606FB03136048996D026801328A42CC
:102CA0000260C0F0738105605B6D9847636A002B1A
:102CB00000F06C81A368012B58D1584A4E49136823
:102CC000D1F854110133B3EB411F13604ED3544973
:102CD000002313600B68013B052B2ED8DFE803F0BF
:102CE00003090E141C2594F849303E2B25D80133D6
:102CF0000EE094F8483003B3013B12E094F84A30F8
:102D00003E2B1AD8013314E094F84930ABB1013BA3
:102D1000394A82F849302BE194F848303E2B0CD8E0
:102D20000133354A82F8483022E194F84A3023B121
:102D3000013B314A82F84A301AE13A4B1A680132B3
:102D4000072A00D101221A601B68374A0B601168FC
:102D5000334801310D29116000F005810E2905D19C
:102D6000013B08BF06230360002313606368032B45
:102D70007BD12E4A20491368D1F894110133B3EB6B
:102D8000411F136071D32A49002313600B68013B74
:102D9000052B51D8DFE803F003090F151D2694F821
:102DA0004C303E2B48D801330FE094F84B30002BC9
:102DB00042D0013B12E094F84D303E2B3CD8013319
:102DC00014E094F84C30BBB3013B0B4A82F84C3012
:102DD000D3E094F84B303E2B2ED80133064A82F8CC
:102DE0004B30CAE094F84D3033B3013B024A82F8CD
:102DF0004D30C2E0200200203000002004060020F8
:102E000024020020A4A4000860050020C0050020C2
:102E10007405002034040020C8040020C8050020E8
:102E2000A4040020CC04002018020020D4050020B7
:102E3000C4050020E0050020564B1A680132072A1D
:102E400000D101221A601B68534A0B601168534875
:102E500001310D29116000F093800E2905D1013B4D
:102E600008BF0623036000231360A36A002B40F011
:102E70008D8003F09BF989E01F4600260096D9F863
:102E80000030474A1B01D3589E42BFF4DDAE009D7F
:102E9000DFF81CB1DFF81CA1009B414AEB1A01933B
:102EA000D9F8003001981B011A445168814257D962
:102EB0003C490968A94205D9D268525D402A01D926
:102EC000413A00E00022D8F80010B2EB910F45D84B
:102ED000002F35D0324A344913449B6803A85B5D08
:102EE000303B03EB4303CA18CB5C02A98DF80830D2
:102EF00053788DF8093093783A468DF80A300123DB
:102F0000FEF7A2FE294B9DF80C20DBF8000033F8F9
:102F1000122004A98DF810209DF80D2033F81220FE
:102F20008DF811209DF80E2033F81230DAF80020C9
:102F30008DF8123033180B2000FB0320002209E02B
:102F4000DBF80000DAF8002033180B2000FB032028
:102F50003A4605A9019B1844FDF7E6FF01359BE7BA
:102F6000013600958BE70133072B04D1012302E0E2
:102F7000FFF704F9FAE60360F8E6FFF7B7F874E73D
:102F80000133072B00D1012303606EE707B0BDE8D2
:102F9000F08F00BFC00400201C020020C4050020E8
:102FA000A4A40008600500205BAC0008D4A40008BD
:102FB000C00500207405002010B5094A044692F8A7
:102FC00048303E2B0BD80CBF3F23023382F84830E9
:102FD000FFF7D4F81CB1BDE8104004F09DB810BD57
:102FE0003000002010B5094A044692F8483063B119
:102FF000012B0CBF0023023B82F84830FFF7BEF8DC
:103000001CB1BDE8104004F087B810BD30000020AE
:1030100010B5094A044692F849303E2B0BD80CBF34
:103020003F23023382F84930FFF7A8F81CB1BDE80E
:10303000104004F071B810BD3000002010B5094AEE
:10304000044692F8493063B1012B0CBF0023023BC8
:1030500082F84930FFF792F81CB1BDE8104004F047
:103060005BB810BD3000002010B5094A044692F844
:103070004A303E2B0BD80CBF3F23023382F84A3034
:10308000FFF77CF81CB1BDE8104004F045B810BD56
:103090003000002010B5094A044692F84A3063B166
:1030A000012B0CBF0023023B82F84A30FFF766F881
:1030B0001CB1BDE8104004F02FB810BD3000002056
:1030C000027808B53F2A0B4B28BF3F2283F84820DF
:1030D00042783F2A28BF3F2283F8492082783F2A3E
:1030E00028BF3F2283F84A20FFF748F8BDE8084090
:1030F000FDF708BD3000002038B50B4B1446DA68E8
:103100000D4682420ED00F2886BF0F22DA60D860AB
:10311000FFF734F80DB103F047FF1CB1BDE83840AC
:10312000FDF748BD38BD00BF3000002010B5074A8C
:103130000446D36843B1013BD360FFF71FF81CB1CD
:10314000BDE8104003F030BF10BD00BF30000020CC
:1031500010B5074A0446D3680E2B08D80133D36054
:10316000FFF70CF81CB1BDE8104003F01DBF10BD07
:103170003000002038B50B4B14461A690D468242C8
:103180000ED00F2886BF0F221A611861FEF7AEFF1E
:103190000DB103F029FF1CB1BDE83840FDF742BD79
:1031A00038BD00BF3000002038B50B4B0D465861CC
:1031B0001C4609B103F000FF63694BB9012229469F
:1031C0000F20FFF799FF012229460F20FFF7D2FFBA
:1031D000BDE83840FDF7FEBC30000020027808B59D
:1031E0003F2A0B4B28BF3F2283F84B2042783F2ACF
:1031F00028BF3F2283F84C2082783F2A28BF3F22F5
:1032000083F84D20FEF772FFBDE80840FDF7F2BCE1
:1032100030000020034A142303FB00239965FDF7C7
:1032200041BD00BF30000020034A142303FB0023EC
:103230001966FDF737BD00BF30000020034B03EBDC
:103240000013C3F84411FDF74DBD00BF300000204E
:10325000034B03EB0013C3F86411FDF75FBD00BF20
:1032600030000020034B03EB0013C3F86C11FDF793
:1032700055BD00BF30000020054B4022184480F8A7
:10328000341003F1340140F2971000F075B900BF1B
:103290003000002037B5012414F0010F14BF39238A
:1032A000002314F0020F8DF8043014BF39230023DB
:1032B00014F0040F8DF8053014BF392300238DF866
:1032C00006300025284601A9013504F009FBAE2D82
:1032D000F8D1FDF7B9FB01340320FDF709FB082CF9
:1032E000DAD10020FEF730FCFEF700FF03B030BD5E
:1032F00037B5134D0446AB6AFBB14208114901A82A
:1033000005F094FC0020FEF71FFCFEF789FC00226C
:10331000104601239DF80410FDF784FD01230022CF
:103320009DF805100620FDF77DFD04F00101490020
:10333000A86AFDF745FB01232B6203B030BD00BF37
:103340003000002054A5000804F00ABB38B504463C
:1033500002F0FAFD08B9012038BD552002F074FED4
:103360000D48082102F09CFE442002F06DFE002C66
:10337000F1D043F21545002402F02CFE013410B9BF
:10338000AC42F9D103E043F215439C42E3D102F091
:10339000DBFD002038BD00BF2C060020F8B5064636
:1033A0000D46144602F0D0FD002834D0552002F01E
:1033B0004BFE194F0821194802F072FEBE2002F0A0
:1033C00043FE0921384602F033FE02F0BDFD144BE6
:1033D0001A683B46222A01D0282A13D15A78197834
:1033E0001B79D009C3F341130933336002F007029C
:1033F0002860181FC3F10C03824041FA03F31A43FB
:10340000226007E00923336097F90130DB0F2B605E
:103410003B7823600120F8BD1C0600202C0600200C
:1034200028060020F8B5A0F10904032C064601D9AE
:1034300000255CE002F052FE02F086FD0028F7D085
:103440002C4F384602F037FE3B782B4A012113609F
:103450002A4A222B0546116001D0282B47D102F0C1
:1034600073FD002843D0552002F0EEFD244F0821C3
:10347000204802F015FEBE2002F0E6FD0921384684
:1034800002F0D6FD3B79C3F3411309339E422ED09F
:1034900002F05AFD58B3552002F0D6FD0821154818
:1034A00002F0FEFD4E2002F0CFFD7F2002F0CCFDA9
:1034B000802002F0C9FD600100F0E00002F0C4FDD0
:1034C00002F042FD02F040FD88B1552002F0BCFD43
:1034D0000821084802F0E4FD482002F0B5FDFA2476
:1034E00002F078FD08B9013CFAD102F02DFD284622
:1034F000F8BD00BF2C060020280600202012002066
:103500001C060020F0B585B000F060FC0C4E0024D5
:1035100001276000012540F0A00000970DF10F0386
:103520002A460021306000F087FC10B9054B1D6071
:1035300002E00134082CECD1024B186805B0F0BD54
:10354000340600203806002013B50B4608490C68E5
:1035500054B10146074800920068012200F06CFC5B
:10356000B0FA80F0400900E0204602B010BD00BF74
:1035700038060020340600202DE9F743134B80461F
:103580001B680E460BB900201DE0114F0C46B946D2
:103590008D18C6EB0801AC4221444FF0010211D056
:1035A0000C4800922346006800F0AAFC0028EAD1EB
:1035B00010233A68002AFCD0013BC9F80000F8D17A
:1035C0000134E6E7104603B0BDE8F083380600207A
:1035D000241200203406002030B5304B87B01A6822
:1035E0000446824258D01860684604F07BFC02A86A
:1035F00004F062FF0121042004F008FE01210420F0
:1036000004F004FE01214FF4003004F00BFE04230B
:10361000ADF8003003251823694621488DF80330A2
:103620008DF8025004F010FC0823ADF80030694614
:1036300048231B488DF803308DF8025004F004FC39
:103640000121184804F06FFF0C23029402A9002402
:103650001448ADF81230ADF80C40ADF80E40ADF89E
:103660001040ADF8144004F0D3FE01210D4804F0E1
:103670002EFF0C48012240F2255104F034FF26238E
:103680008DF8043001A801238DF805408DF806401F
:103690008DF8073004F030FA07B030BDC8060020BE
:1036A000000801400044004030B40E490B680D4A48
:1036B0007F2BFBD80C4B0D4D1C68C0B2611C7F29C1
:1036C000196088BF0021285588BF196072B6136839
:1036D0000133136062B6012240F2277130BC044806
:1036E00004F001BFCC060020C006002040060020E8
:1036F0000044004010B5441E14F8010F10B1FFF74C
:10370000D3FFF9E710BD0000024B1868003018BF66
:10371000012070473C06002030B50C4B1A689AB166
:103720000B490C4D0A68541CB4F5807FAA5C0C60F0
:1037300008BF0024D2B208BF0C6072B61968013904
:10374000196062B602600122104630BD3C060020BE
:10375000D0060020D4060020024A1368002BFCD1BA
:10376000704700BFCC06002038B540F225512448F0
:1037700004F0E5FEC8B140F22551214804F0FFFEF7
:103780001F4804F0CCFE1F4B1A68FF2A0DD81E4AB2
:103790001E4D1468C0B2611CFF291160285584BFFA
:1037A000002111601A6801321A6040F22771144832
:1037B00004F0C5FE10B340F22771114804F0DFFE9B
:1037C000134B1A689AB1134A134C1168481C80288D
:1037D000106008BF0020615C08BF10601A68C9B2A1
:1037E000013A1A600648BDE8384004F094BE40F241
:1037F0002771BDE83840024804F075BE38BD00BFEF
:10380000004400403C060020D4070020D4060020DD
:10381000CC060020C406002040060020074A0023F2
:1038200030B5012898BF022011461C461568002DAE
:10383000FCD0013383420C60F8D130BD2812002047
:10384000F7B5214D01A804F04DFB0121042004F03F
:10385000DDFC01240227102601A92846ADF804400A
:103860008DF806708DF8076004F0EEFA214604200A
:1038700004F0CCFC01A92846ADF804708DF8067060
:103880008DF8076004F0E0FA2146042004F0BEFC45
:1038900001A92846ADF804608DF806708DF8076020
:1038A00004F0D2FA22462146284604F029FB22469B
:1038B0003946284604F024FB22463146284604F0C7
:1038C0001FFB03B0F0BD00BF00080140F7B500F0DA
:1038D000CBFFFFF741FFFFF717FF002800F0B18093
:1038E0005E4E5F4D01A8FFF717FF002800F0A9808A
:1038F000019A01230A2A3360584F40F096802A68C3
:10390000584C0023A354002A00F08C80544A1360C2
:1039100023782E2B03D16378002B00F0948052483B
:1039200000F078FF4F4800F075FF504800F072FF3C
:1039300000F09AFF02224E494A4805F0BAF90028E1
:1039400000F0818005224B49464805F0B2F9002875
:103950007BD002224849434805F0ABF9002876D0D5
:103960000A2246493F4805F0A4F940B90F224449CC
:10397000444805F0B3F901237B6004206AE0032288
:103980004149384805F095F930B91F223F49404870
:1039900005F0A4F905205DE005223E49314805F017
:1039A00088F958B902223C493C4805F082F908B927
:1039B000022300E00123BB6006204BE005223849CA
:1039C000284805F076F930B90F223449354805F01A
:1039D00085F907203EE008223349224805F069F9BD
:1039E00030B93F223149324805F078F90A2031E0F8
:1039F000092230491B4805F05CF930B90F222E49E5
:103A00002E4805F06BF9082024E004222C491548C3
:103A100005F04FF9E8B93F222A492B4805F05EF935
:103A2000092017E000F020FF5CE70D2A3FF45AAFB1
:103A30002B68FF2B3FF656AF591C29600949CA5421
:103A400050E7002008E0012004E0022002E003200B
:103A500000E0FF200023237003B0F0BD2C120020F3
:103A6000E0080020DC070020E4B10008E6B100080F
:103A7000EAB10008EDB10008F3B10008F6B10008A2
:103A8000E60700206812002001B20008DF070020CE
:103A90004812002005B200080BB20008E107002020
:103AA0000EB20008B812002014B20008E40700208B
:103AB000C81200201DB20008E507002038120020BF
:103AC00027B20008E00700207812002073B50446F2
:103AD00005F0E7F80546144800F09CFE264625440C
:103AE000AE4211D016F8012BA2F120035E2B03D8B1
:103AF000104600F069FEF3E70C49684605F096F8B9
:103B0000684600F087FEEBE7094800F083FE00F00E
:103B1000ABFE2046FFF7EEFD0648FFF7EBFDFFF793
:103B20001BFE02B070BD00BF2CB2000831B200080D
:103B300038B20008E7B1000873B5002201210E4831
:103B400004F0DEF90520FFF769FE0C4E0122114654
:103B5000094804F0D5F9354600233360322401A822
:103B6000FFF7DAFD0028F7D12B68002BF7D0013CD6
:103B70002860F4D102B070BD000801402812002076
:103B800000B5094BA1B0002283F83C205A600B46D7
:103B90000246064901A805F049F801A8FFF796FF7B
:103BA00021B05DF804FB00BF2C12002044B20008D5
:103BB000034B0022034883F83C205A60FFF786BF7E
:103BC0002C12002051B2000807B54FF4E13000F08C
:103BD000CAFEFFF735FE4FF4E130FFF7FDFC00228F
:103BE0001021144804F08CF900220121114804F03E
:103BF00087F90520FFF712FE012211460D4804F057
:103C00007FF93220FFF70AFE01221021094804F053
:103C100077F901A8FFF780FD10B1019800F0D4FDFD
:103C200001A800F001FE0028F3D00198FFF73CFD49
:103C3000EFE700BF0008014008B50B4B1A6892B9C6
:103C400001224FF4E1301A6000F08DFE074800F0C9
:103C5000E1FDFFF7F5FD4FF4E130FFF7BDFCBDE8F6
:103C60000840FFF769BF08BDD807002055B200081B
:103C70001FB5684604F0FEF94BF6FF720023ADF85D
:103C80000430ADF808304FF48063ADF80A30094CC9
:103C90004FF48043ADF80C30074B20460121ADF8BE
:103CA0000620009304F0F4F96946204604F078F900
:103CB00004B010BD00540040A086010010B50A4CAD
:103CC0000121204604F0FCF92046012104F01EFAEF
:103CD0002046002104F01AFA204604F047F9BDE816
:103CE0001040FFF7C5BF00BF0054004070B5064646
:103CF0000D4643F201043146084804F013FA28B98E
:103D0000013CF8D1FFF7DAFF204670BD2946034891
:103D100004F008FA0028F3D0012070BD00540040E0
:103D200038B5054643F201042946064804F0FAF97D
:103D300028B9013CF8D1FFF7C1FF204638BD01206A
:103D400038BD00BF00540040F8B506460F461B487A
:103D5000012114461D4604F0A7F91948FFF7E0FFBA
:103D600010B30DB1002100E00121144D134804F0FF
:103D7000B3F928460022F1B204F0BFF91148FFF769
:103D8000CFFFA0B110482B8BFFF7CAFF90B1FEB256
:103D900024B1C7F30721284604F0AAF92846314682
:103DA00004F0A6F90020F8BD4FF0FF30F8BD6FF029
:103DB0000100F8BD6FF00200F8BD00BF00540040E4
:103DC00001000010020000108000001037B5184BF1
:103DD0001D6855BB012401A81C6004F083F821462E
:103DE0004FF4001004F01EFA2146082004F00EFAE9
:103DF0002146082004F00AFA21464FF4001004F08E
:103E00001DFA29464FF4001004F018FAC023ADF84B
:103E100004301C238DF8073001A9032305488DF8D1
:103E2000063004F011F8FFF723FF03B030BD00BFE8
:103E3000E4080020000C01402DE9F041069E1D46DB
:103E4000741E634263418046FFF77EFF04460028EC
:103E500037D125492548FFF749FFA0B3244F012159
:103E6000384604F021F92348FFF75AFF78B3384663
:103E700001225FFA88F104F040F91F48FFF750FF74
:103E800048B33B8B013DB44214D00134A64207D164
:103E90000021174804F020F90121154804F010F919
:103EA0001648FFF73DFFD0B1114804F023F905F89B
:103EB000010FE8E701210E4804F00EF90020BDE8EB
:103EC000F081BDE8F0816FF00300BDE8F0816FF094
:103ED0000400BDE8F0816FF00500BDE8F0816FF0EF
:103EE0000600BDE8F08100BF040000108000001053
:103EF00000540040010000100200001040000010BB
:103F000038B51C460023FFF71FFFF0B90F48FFF735
:103F100007FFB8B1049BE518AC420DD014F8011BA3
:103F20000B4804F0E5F80B490848FFF7DFFE0028CE
:103F3000F2D16FF0030008E00121054804F0C0F859
:103F4000002038BD6FF0020038BD38BD8000001081
:103F5000005400400400001070B52C4A2C4C516AEB
:103F60002368994205D8956AAB4202D2D66B294D97
:103F700008E0D16A254D8B420FD32E6BB3420CD291
:103F8000EE6B254D2EB1591A2E6800FA01F131431E
:103F900002E0296840EA410129601268032A09D138
:103FA000A3F11102032A2DD81C4990400A6810433E
:103FB000086027E0052A25D1A3F11402032A06D8B8
:103FC000154DA3F1080200FA02F12A6807E0A3F1F7
:103FD0001801032906D8124D00FA02F229680A4393
:103FE0002A6001E02F2B0DD803F007060122D90823
:103FF0000C4DB24010B1685C024302E0685C20EAFC
:1040000002026A540133236070BD00BF0C09002016
:10401000F8080020500900207009002068090020DD
:1040200060090020EC08002007B501A803F05AFF42
:104030000121082004F0EAF80823ADF80430022337
:104040008DF8063004230DEB030104488DF807308A
:1040500003F0FAFE03B05DF804FB00BF000C014062
:1040600070B5254C2368002B31D0244A244B1168AD
:10407000022911D003292CD11D681968C943C9B27E
:10408000B1EB152F1FD11968C9B219601D490D6810
:10409000196841EA052114E01D681968C943C9B2CD
:1040A000B1EB152F0BD048F2EE71174D2E688E42F2
:1040B00009D10B2111601968C1F307212960196822
:1040C000C9B2196005E000200023236070BD1846C6
:1040D00070BD12680C4D02702A680C49A0F80120CE
:1040E0001A68A0F803200A68427100221A600120B1
:1040F0002A600A60E8E700BF740900200809002070
:10410000F4080020FC080020580900205C09002069
:104110002DE9F84F9F4D08219F4803F0EBFE2A68D8
:10412000002A40F022829D490B680E461BBB9C4A28
:1041300008B913681CE012689AB101220A60994913
:104140000A6099490B6099490B6099490B6099493C
:104150000B6099490B60994BFF211960984B1A70BD
:1041600003E24FF6FE71974A13688B4200F2FD811D
:1041700001331360F9E18B4FD7F800C0BCF1000F99
:104180004DD08F4C58B123780133DBB2E92B23702B
:1041900040F2BF80824B0A601A602270B9E0804A08
:1041A00013689046A3F11F010A2903D82278063A22
:1041B000042A1DD9A3F15E02532A07D82278A2F15E
:1041C0002E012B2916D9173A162A15D9A3F13C022C
:1041D0000F2A03D822783C3A0F2A0FD9283B162BF6
:1041E00003D82378133B0C2B0AD90021316008E057
:1041F000754906E0754904E0754902E0754900E03B
:10420000754933681BB14422744804F007FC6B4ABB
:10421000002313600122C8F8002023706DE0624B78
:104220001A681C46002A6AD06C4B002847D0634AA3
:104230005F6B116896468F420DD19A6B012A0AD1A5
:10424000574A59691268914218D899698A4215D813
:10425000C3F838C061E0DFF86881186898F800207A
:10426000012802F10102D2B288F80020DFF86CC107
:1042700007D0E92A51D97A1E91421AD0002333601F
:1042800077E00B2A45D90A29F3D9494F4A1CCCF8C3
:1042900034203A68A1F10B0E42EA0E223A60DCF8B3
:1042A0002C20114401310A22CCF8301088F800206B
:1042B00005E09B6B002BE1D1CEF800702DE0196872
:1042C000464A0329364FDFF8F8E040F08D803B483E
:1042D0000168102940F088803B68053B072B00F2FD
:1042E0009D809EF80030A3F13C0EBEF10F0F45D823
:1042F000002323601123036001233B6009E020B900
:10430000274A13680133136003E001221A602C4B23
:104310001A703368002B00F02881304B274A5F6BFE
:104320001268974240F021819A6B002A40F01D816B
:104330002B4C1E4AD4F800E011688E4529497ED1E5
:1043400020480068B0F5966F79D2086801301B6884
:104350000860012B75D10968013901297ED8194BF4
:10436000002119602B68002B40F0D78000233360B8
:1043700013600B4A1360124A1370F6E00F3B0A20D9
:10438000D1620F2B4FF020011060116351633FD8B1
:1043900001203EE074090020000C01405409002077
:1043A0006C09002078090020E8080020700900202E
:1043B000500900206009002068090020F80800204A
:1043C000040900200009002068B2000834B3000886
:1043D000ACB2000878B30008F0B200080C09002065
:1043E00048020020640900203A68586860499042F9
:1043F00019D95B695E499A4210D38B699A420DD8EC
:104400009EF80030CA69934208D30A6A934205D8DD
:104410000020FFF7A1FD002323606DE70023336038
:104420008EF8003068E788688242E2D89EF800C0C3
:10443000C8688445DDD309698C45DAD8A8E700202F
:1044400085E7052B03D10968012907D187E70A2BE6
:1044500001D0292B02D10968C90780D40121022B80
:10446000DFF8349129604348DFF83081DFF830C14C
:104470001BD14149002F70D1DFF818A1DAF80030C4
:10448000B3F5E16F0ED20B68DFF8F4900360D9F852
:104490000030C2F800E043F00103C9F80030CAF868
:1044A00000705AE0C9F8007057E0052B29D1334B52
:1044B0001F7893F801B007F00F0193F802A081EA8A
:1044C00017110BF00F07794081EA1B110AF00F0753
:1044D000B94218BF0021DF7818BFC9F80010197958
:1044E0008AEA070793F8059087EA010399451CBFFC
:1044F00000232B602249234B0F681B683B430B6052
:104500000523C8F800300368CCF8003011681E4B52
:1045100019601E4B19681E4B23E71068DFF854C062
:1045200086451C49DFF850E00FD1DEF80070DCF85A
:1045300000309F4209D140F6C9070B68BB429FBFBC
:104540000F4F3B6843F001033B60DCF80030206014
:10455000CEF8003000230B6008E70223C8F80030D3
:104560000368CCF800300B60D0E72868BDE8F88F0E
:104570000C090020500900204C020020EC0800200B
:104580005C09002060090020F40800206809002070
:10459000FC08002000090020740900200809002000
:1045A00058090020FBF766BE10B5104CA01CFBF7A5
:1045B0006FFE2346C0B15A88A488A24238BF5C80EF
:1045C000DA885988914284BF08494A80944209D2C6
:1045D0005988121B091B490191FBF2F2D2B21F2A22
:1045E0001A7001D91F221A7010BD00BF7C0900206B
:1045F00038B540F6FF73114C0025E380104BA580C1
:104600001B68CBB10F4B984216D90222211DE12025
:10461000FEF79AFF0222A11DE320FEF795FF4FF659
:10462000FF73A2889A42E28808BFA5809A4202BF1F
:1046300040F2FF32014BDA8038BD00BF7C09002018
:1046400038060020FF00020008B50A4B1B680BB9B2
:10465000002008BD02220849E120FEF78DFF002856
:10466000F6D002220549E320FEF786FF003018BF8E
:10467000012008BD380600208009002082090020A2
:1046800013B5FBF7F7FD0A240DF10600FBF700FE5A
:1046900028B90A20FCF71EF9013CF5D105E0BDF868
:1046A0000620044B9A80FFF7CFFF024B988802B098
:1046B00010BD00BF7C09002013B5FBF7DBFD0A2409
:1046C0000DF10600FBF7E4FD28B90A20FCF702F91A
:1046D000013CF5D105E0BDF80620044BDA80FFF778
:1046E000B3FF024BD88802B010BD00BF7C09002088
:1046F000FBF764BD30B5314B87B01A68044682427F
:104700005AD01860684603F0EDFB02A803F0D4FE0F
:104710000121042003F07AFD0121042003F076FD3D
:1047200001214FF4804003F071FD4FF40073ADF8A8
:10473000003003251823694621488DF803308DF891
:10474000025003F081FB4FF48063ADF800306946FE
:1047500048231B488DF803308DF8025003F074FB9A
:104760000121184803F0DFFE0C23029402A9002463
:104770001448ADF81230ADF80C40ADF80E40ADF86D
:104780001040ADF8144003F043FE01210D4803F042
:104790009EFE0C48012240F2255103F0A4FE252381
:1047A0008DF8043001A801238DF805408DF80640EE
:1047B0008DF8073003F0A0F907B030BD100A0020D3
:1047C000000801400038014030B40E490B680D4A22
:1047D0007F2BFBD80C4B0D4D1C68C0B2611C7F2990
:1047E000196088BF0021285588BF196072B6136808
:1047F0000133136062B6012240F2277130BC0448D5
:1048000003F071BE140A0020080A00208809002065
:104810000038014010B5441E14F8010F10B1FFF725
:10482000D3FFF9E710BD000030B50C4B1A689AB100
:104830000B490C4D0A68541CB4F5807FAA5C0C60CF
:1048400008BF0024D2B208BF0C6072B619680139E3
:10485000196062B602600122104630BD8409002052
:10486000180A00201C0A0020024A1368002BFCD101
:10487000704700BF140A002038B540F22551244883
:1048800003F05DFEC8B140F22551214803F077FEE8
:104890001F4803F044FE1F4B1A68FF2A0DD81E4A1A
:1048A0001E4D1468C0B2611CFF291160285584BFD9
:1048B000002111601A6801321A6040F22771144811
:1048C00003F03DFE10B340F22771114803F057FE8C
:1048D000134B1A689AB1134A134C1168481C80286C
:1048E000106008BF0020615C08BF10601A68C9B280
:1048F000013A1A600648BDE8384003F00CBE40F2A9
:104900002771BDE83840024803F0EDBD38BD00BF57
:1049100000380140840900201C0B00201C0A0020E4
:10492000140A00200C0A00208809002010B5064C4B
:104930000B4602464FF48071204604F0C7FC204627
:10494000BDE81040FFF766BF200B00200FB407B58D
:1049500004A951F8040B0191FFF7E8FF03B05DF8DB
:1049600004EB04B07047FFF7C5BE000001460148E4
:10497000FFF7ECBFBCB30008044B186828B1402215
:10498000034940F2FF10FEF7F7BD704738060020DC
:1049900034130020044B186828B14022034940F228
:1049A0003F20FEF7E9BD7047380600207413002051
:1049B00010B5524C01214FF0804003F025FDFFF768
:1049C000A7FB2368012B0CD940F6A6614C4A13685B
:1049D00001338B42136004D14A4B0121196000233B
:1049E0001360494A13680133EA2B136004D1474B23
:1049F0000121196000231360454A13680133962B87
:104A0000136003D100231360FBF76EFD414A136866
:104A10000133962B136004D13F4B01211960002311
:104A200013603E4A136801330F2B136004D13C4BD3
:104A3000012119600023136043F69821394A136855
:104A400001338B4201D0136010BD374B0021116040
:104A500001221A60236813442360344B1868104401
:104A6000186018682D2809D13149324B08681C6834
:104A7000844236D0096819602F4B31E0186831281C
:104A800001D12E4B2CE01868322801D12C4B27E0A5
:104A90001868332801D12B4B22E018683C281BD121
:104AA0001960234B186801301860274802601A68A3
:104AB0003C2A16D11960254B1A6801321A601A680F
:104AC000182A0ED11960224B1A6801321A601A682E
:104AD000072A06D1196004E01B681E2B01D11D4B6B
:104AE0001A601D4B1A683AB11A68013A1A601B68BD
:104AF00013B91A4B01221A6010BD00BF280C002008
:104B00004C0C00205C0C0020540C00206C0C00208D
:104B1000200C0020740C002028120020400C0020E3
:104B200024120020300C00202C0C0020680C0020E7
:104B3000700C002058020020480C0020640C00205B
:104B4000380C0020600C00203C0C0020580C002089
:104B5000340C0020440C002050020020240C0020C3
:104B60002DE9F04F97B003F06FFD03F0E7FD012151
:104B7000084603F04BFB834E0121834803F0C6F93E
:104B800008234FF4E130F380FFF7EDFEFFF74CFA16
:104B900001F0CCFA01F0EEFA0520FBF7B3FE0EA807
:104BA00003F0E6FB0121084603F03CFB0023ADF8CF
:104BB0003E30ADF83A300523ADF83C3040F21F33BB
:104BC0000EA94FF08040ADF8383003F043FB0122CE
:104BD00011464FF0804003F001FC1C238DF830306B
:104BE00001240F230CA88DF831308DF832308DF868
:104BF000334002F081FF21464FF0804003F0CBFBB1
:104C0000FBF7C6FBFBF7E2FB02F02EFD01F030FCE8
:104C1000FEF778FCFBF7F2FB18B1FBF7A9FBFEF7F8
:104C2000D3FF5A48FFF7F6FD5948FFF7F3FD5948FF
:104C3000FFF7F0FD5648FFF7EDFD5748FFF7EAFD97
:104C4000564F5748FFF7E6FD5148FFF7E3FD3B6835
:104C50000BB1544800E05448544DFFF7DBFD4C487D
:104C6000FFF7D8FDFEF770FB2B68002B64D050488F
:104C7000FFF7D0FD4648FFF7CDFD2B6823B1042296
:104C80004C490020FEF760FC4A4C4B482168FFF776
:104C90005DFE236823F47F0222F47F42002A51D173
:104CA000A3F582314548A1F5807181424AD8190C9B
:104CB00030311B0A303331702E21B3707170327174
:104CC00001F062FB2068FDF76BFB01F0FBFF206841
:104CD00001F03CF820683A4B984207D901F02EFDCC
:104CE000206801F0ABFC2068FFF782FC2268354B9E
:104CF0009A4201D902F09AFB2B681BB32268324B0F
:104D00009A4210D94022314940F2FF10FEF71CFCB4
:104D1000C0B1264B1B68ABB140222D4940F23F2069
:104D2000FEF712FC0EE02B49284803F0B2FF2A4997
:104D3000274803F0AEFF05E02848FFF76BFD144855
:104D4000FFF768FDFFF7D4FCFBF798FB01F0FAF8DA
:104D500001F03EFDFCF764FF2B68002B00F08D8016
:104D6000144C1F4E2368B34200F0878031461D4823
:104D7000FFF7ECFD0D4B26601B68BBBB1A48FFF725
:104D8000F5FD3AE00813002000023000DDB3000812
:104D9000E7B10008FCB3000819B40008680200205D
:104DA00023B4000829B4000837B4000838060020EE
:104DB00046B400085C02002057B40008000101005E
:104DC000FF000200FF010200FF0502003413002073
:104DD0007413002078B4000882B4000889B4000875
:104DE000000602009BB40008BFB40008042221465C
:104DF0000020FEF7C1FB0028C0D001F0F1FA10B985
:104E00009C48FFF7B3FDFDF797FC10B99A48FFF7F0
:104E1000ADFD01F085FF10B99848FFF7A7FD00F040
:104E2000E7FF10B99648FFF7A1FD01F0AFFC10B9FC
:104E30009448FFF79BFD01F029FC10B99248FFF759
:104E400095FDFFF701FC10B99048FFF78FFD02F0C8
:104E50002DFB10B98E48FFF789FD2B68002B00F061
:104E60004787FFF789FD002800F04287FFF792FD92
:104E7000002800F03D87874B2360874B0122874C39
:104E80001A602568114610460335FCF74CF8236874
:104E90009D4219D90CA8FFF7E3F80028F7D00022AB
:104EA00011460120FCF73FF80120FBF721FD0CA87B
:104EB000FFF7D6F8002211461046FCF734F801F04F
:104EC000D3F908B101F08CFA002211461046FCF724
:104ED0002AF8FEF7B1FE724B1B680BB101F016FC0D
:104EE0003B680BB101F0F4FB4FF00009C846FF2608
:104EF0006C4F07960696CDF82490CDF820900424A8
:104F0000CDF81490654BD3F800B0059B83B3089B94
:104F1000C3EB0B03052B14D9FBF770FA88B1624879
:104F2000FFF778FC6148FFF775FC614B002261498F
:104F300061485A6083F83C20FEF722FECDF820B08D
:104F400016E0099BC3EB0B03052B11D902F0A4FB60
:104F500070B15A48FFF75EFC5448FFF75BFC544BB6
:104F600000225A6083F83C20FEF722FECDF824B0E0
:104F7000B8F1000F07D0B8F1010804D1424641460C
:104F80004046FBF7D0FFFEF7A1FC0928054640F09C
:104F90002783474D95F84C304E2B00F0958011D863
:104FA000442B00F0448206D8412B00F08D82432B25
:104FB00000F0AD8266E3472B00F007834D2B00F035
:104FC000BD825FE3542B00F0AA8105D8522B25D077
:104FD000532B00F0688155E36E2B00F04381742B56
:104FE00000F0CF82612B40F04D83022105F14D008E
:104FF000FBF791F902210B9005F14F00FBF78BF9BC
:105000000221824605F15100FBF785F902210A9041
:1050100005F15300FBF77FF92949CAE2022105F1A6
:105020004D00FBF778F9062800F22C83DFE800F04A
:10503000060B1018041B1E00042623E3FFF720FBB9
:1050400001F0EAFF1EE3FFF737FB01F0EDFF19E384
:1050500001F00AF9002800F0158301F0C1F911E30D
:105060000122184BE1E1FEF715F90AE302F0B2FA6A
:1050700008E300BFC7B40008D0B40008E6B40008D5
:10508000FFB4000818B5000832B5000844B50008A0
:1050900056B5000800060200480C0020280C00202D
:1050A00020120020300000206CB50008E7B1000895
:1050B0002C120020A5B50008B0B50008BAB500084C
:1050C000F4130020240C0020022105F14D00FBF711
:1050D00022F90221824605F14F00FBF71CF902215B
:1050E0000A9005F15100FBF716F90A9BAAF1030A91
:1050F00043EA0025BAF11C0F00F2C482DFE81AF07F
:105100001D003300C2023C004B004F005B006C00EE
:1051100078008100850089009000C202C202C202AC
:105120009900C202C202A000C202A6005E00630093
:1051300066006900C2022B00AE00BB6A9D4200F00F
:10514000A1822846BD62FDF749F8BB6A002B14BF57
:105150000C24142496E2FB6A9D4200F093822846B8
:10516000FDF73CF88EE23B689D4200F08B82002107
:105170002846FDF777FB84E27B6933B1C44B0021FD
:10518000FF2208461A60FEF70FF801220021284688
:10519000FDF7B2FF42E02846FDF71CFB71E2BC4B75
:1051A000FF221A6015B10021012001E0294628469E
:1051B000FDF7FAFF66E22946042001E029460020B7
:1051C000FEF75AF85EE229460120F9E72946022057
:1051D000F6E729460320F3E7FB699D4200F052827F
:1051E00000212846FDF776FBAA4B00221A6048E210
:1051F0007B689D4200F0468200212846FDF702FBB5
:105200003FE22846FDF712FB3CE22846FDF71CFB77
:1052100038E2012200212846FDF7ACFF022431E2EA
:10522000BB689D4200F02E8200212846FDF784FBDA
:1052300028E2E8B2EB0548BF404201F087FD21E2D9
:10524000284601F03BFA0122934BEEE0284601F09C
:10525000B5FA924A01231360914AF3E12846FDF71B
:10526000ADFA0FE2022105F14D00FBF754F80221DF
:105270000A9005F14F00FBF74EF80221824605F136
:105280005100FBF748F80A9B0146002B40F0FA81D9
:10529000BAF13F0F00F2F6810F2800F2F381504679
:1052A000FDF73AFAEEE1022105F14D00FBF733F884
:1052B0000A2800F2E781DFE810F00B00E501E501C4
:1052C000E5010E00120016001A001E0022002A003E
:1052D00001217448D3E1734801F052FDD2E17148D5
:1052E00002F018F9CEE16F4802F026F9CAE16D48E4
:1052F00002F038F9C6E16B4802F050F9C2E13F22F2
:105300006849694803F0EAFCFFF736FBBAE13F223F
:105310006449664803F0E2FCFFF73CFBB2E102217E
:1053200005F14D00FAF7F7FF002840F0AB8195F842
:105330004F206421A2F1300395F8502095F858C011
:10534000303A4A434FF47A7101FB032295F8511029
:105350000A23303903FB012195F85220ACF1300CBF
:10536000303A0A4495F85310DFF850A1A1F130000B
:1053700095F85410CAF81C20303903FB001195F839
:105380005500CAF81810A0F1300E95F8560002F238
:105390006C72303803FB0E0095F857E00131AEF126
:1053A000300E03FB0ECE95F85AC0CAF810E095F8FF
:1053B00059E0ACF1300CAEF1300E03FB0ECECAF862
:1053C0000CE095F85BE095F85C50AEF1300E303DA6
:1053D00003FB0E53CAF81400CAF80830FAF772FF3C
:1053E000334BCAF820001B68504613B1083001F057
:1053F0008FF8304ADAF810301268934207D12E4AFB
:105400002E491268C968914218BF042400E00424A0
:105410002B4ADAF820101160264A1360DAF80C20C3
:10542000254B1A60DAF80820264B1A602AE195F815
:105430004D30022105F14E000A93FAF76CFF0A9BEA
:105440008246432B40F01E81022105F15000FAF7FD
:1054500062FF02218DF8380005F15200FAF75BFF78
:1054600002218DF8390005F15400FAF754FF8DF848
:105470003A00BAF1000F03D10EA8FDF721FE01E1B9
:10548000BAF1010F40F0FE800EA8FDF7A7FEF9E08B
:10549000600200206C0C0020600C0020640C0020D6
:1054A000380C00207B1200203413002074130020DD
:1054B00068020020580C0020700C00200813002007
:1054C000340C0020680C002095F84D30022105F1C5
:1054D0004E000A93FAF71FFF0A9B8246442B0CD01A
:1054E000462B40F0CF80022105F15000FAF713FF60
:1054F00001465046FDF798FEC4E0022105F1500038
:10550000FAF709FF01465046FDF784FEBAE095F828
:105510004D30022105F14E000A93FAF7FCFE0A9B7A
:105520008246442B40F0AE80022105F15000FAF78C
:10553000F2FE01465046FDF781FEA3E095F84D309E
:10554000022105F14E000A93FAF7E5FE0A9B824616
:10555000442B0CD0462B40F09580022105F15000E1
:10556000FAF7D9FE01465046FDF77CFE8AE002219B
:1055700005F15000FAF7CFFE01465046FDF768FEF0
:1055800080E0022105F14D00FAF7C5FE02210B90E3
:1055900005F14F00FAF7BFFE0221824605F15100E6
:1055A000FAF7B9FE02210A9005F15300FAF7B3FEAB
:1055B00086490B9B0A9A01EBC3050AEB02226A603B
:1055C00041F8330000F014FC5CE095F84D30542BAA
:1055D00058D195F84E30732B54D101F099F950E021
:1055E000072831D10A220EA9794803F009FC0146A7
:1055F000784801F0F3FB784B1B6813B1754800F055
:1056000087FFDFF830A2754DDAF800302A699A4238
:1056100004D1734BEA681B689A4202D001F046FD40
:1056200004242A6A6F4B1A602B69EA68CAF80030B2
:105630006B4B1A60AA686C4B1A601B686B4AC3F507
:105640006E63023313601DE0042810D101F0F0FDF9
:10565000674A68490EA803F0E9FA65496648FFF70A
:1056600075F901210EA8FDF753FA2C460AE00A2825
:1056700008D162496248FFF769F960480121FDF7E6
:1056800047FA04247B6A13B37B6903B3FEF78CFFEC
:10569000E8B15C4D5C496A880B6802F110009842E1
:1056A00002D310339A4202D90A6001F0ADFC574A86
:1056B00028781368411C994202D30133984206D9D5
:1056C0001060002211464008FDF716FD0224059BDC
:1056D0004BB94F4B1B68DBB14E48FFF79BF84E4868
:1056E000FFF798F810E04D4B1A686AB9484A01254F
:1056F000526862B14A481D60FFF78CF84648FFF7D0
:1057000089F8484B1D6002E00123059300E00595F0
:105710003048FAF77FFE00283DD0012100220846DC
:10572000FBF701FC2C4B1B6813B12A4800F0F0FE7C
:10573000DFF80081294DD8F800302A699A4204D157
:10574000274BEA681B689A4202D001F0AFFC0424A0
:10575000296A244B28691960214AEB68C8F80000BF
:10576000DFF884E01360AA68D5F818C0CEF80020EE
:10577000D5F81CE00392019002936B692A480093CC
:1057800050F821100CF101030EF26C722748FFF75C
:10579000DDF84FF03208264B1B68002B70D00E4B03
:1057A0001B68002B69D00B4800F000FF002864D074
:1057B0000A49204B08691B6898423DD1084BCA68CA
:1057C0001B689A4218BF042437E000BFB4130020BE
:1057D000B8120020101300206802002008130020D7
:1057E000700C0020340C0020680C002050020020B7
:1057F00068120020EAB50008F0B50008C8120020C1
:1058000008B600087C090020540200206002002035
:105810002C1200201DB60008E7B10008500C002033
:105820002CB60008240C0020000000203FB6000821
:10583000480C0020580C002004240D6A954B964A11
:105840001D60964BDFF87CE21860CB68D1F818C079
:1058500013608A68CEF80020D1F81CE00392019012
:1058600002934B698E4900930EF26C720CF10103A6
:1058700051F825108B48FFF769F88B4B00221A600E
:105880007B6A43B17B6933B1884D2B681BB1FEF74E
:1058900089FE00232B60864D2B688BB1854B5B689E
:1058A00043B1002101220846FBF73DFB01F07EFADF
:1058B0004FF0320840F6D86200232B607E4B1A600E
:1058C0007E4B1A68002A6DD00024DFF8D0A11C603E
:1058D000DAF800207A4B704D1A612A68DA60794A4A
:1058E00012689A606B4A11680A92196201F0DEFB35
:1058F0000A9A3C201268DAF80030296800FB03138A
:10590000B96A204600F0BCFAE0B1B86AB0FA80F09B
:105910004009B862FCF762FCBB6AA34214BF0C24C6
:10592000142401F031FB684BDAF80020996A6748CB
:105930002B68674D002914BF294601466548FFF7CB
:1059400005F800E00446534BDFF850A1524D1A68A9
:10595000DAF8003029683C2000FB0313F96A0120C3
:1059600000F08EFA98B1F86AB0FA80F04009FCF7BE
:1059700035FC5648DFF858E1F96ADAF800200029CA
:1059800014BF714601462B685348FEF7DFFF4CB940
:105990002C680523B4FBF3F303EB83039C4214BF91
:1059A000012404244D4A1368ABB1002313601A4646
:1059B000394DD11991F83400984209D9D5F800E051
:1059C000BEFBF0F100FB11E1002904BF03461646BF
:1059D0000132052AEDD1424B1A6842B100221A6009
:1059E000404B1B681BB1404B186800F08DFE3E4BCE
:1059F0001B68C3B13C4A002313603A4B1B6883B158
:105A000000F084FE394B10F0010F394A4FEA500183
:105A1000069008BF1A463748FEF798FF01F014FBBE
:105A200001E0FF230693344B1A68BAB100221A60D2
:105A3000324B1B6883B100F04BFE2C4B10F0010F72
:105A40002B4A4FEA5001079008BF1A462C48FEF730
:105A50007DFF01F0F1FA01E0FF230793FF2E6CD0E8
:105A6000BD1995F83910022906D82648FEF76EFFB1
:105A700095F839303B636AE0042E45D1069BFF2B35
:105A800002D1079BFF2B68D01846FDF731FC4FF081
:105A9000FF3962E0340C0020700C0020580C00200C
:105AA0000000002068B60008480C00205C0C0020B4
:105AB000240C00202C120020500200203C0C00205E
:105AC00008130020680C00203000002098B7000860
:105AD00085B7000894B60008B3B60008440C00204F
:105AE000640C002020120020380C0020E9B10008CE
:105AF000DAB30008DCB60008600C00206802002061
:105B0000F8B6000810B70008022E26D18348FEF729
:105B100081FE8348FEF77EFE824A0EA8D169936912
:105B200001F26C710091013352697F4903F07EF8F4
:105B300001210EA8FCF7ECFFE1E0B9F1000F0CD059
:105B4000B9F1FF3F06D13B6A3BB97B6A2BB10BF140
:105B5000050902E0D94540F2D08034B1734B2246AA
:105B60001868734B1968FCF74BFB724B1A681AB133
:105B700000221A60FCF7FCFF6F4B1A682AB1002262
:105B80001A606E4B1868FCF7EBFE00F049FBFF282B
:105B9000064600F0BF80002211460120FBF7C3F942
:105BA000132E00F2B480DFE806F00EB22125292D75
:105BB00031363A425F63676B6F738491770A4FF0B7
:105BC00032080426A6E0B86A4FF03208B0FA80F036
:105BD0004009B862FCF702FBBB6AFF26002B14BF2A
:105BE0000C24142401F0D0F9FFF78CB90120FCF744
:105BF0005DFE86E00120FCF745FE82E00120FCF717
:105C000089FE7EE00120FCF773FE7AE0474B1A68BC
:105C100042B9172212E0454B1A68162A0AE0444B93
:105C20001A6812B11A68013A08E03B2206E0404BBC
:105C30001A683A2A96BF1A68002201321A603F4B4E
:105C400000221A603E4B1B68002B5AD0374B354858
:105C50001B680361364B1B68C360384B1B6840F8F8
:105C6000083F00F055FC4CE00120FDF7BBF939E09E
:105C70000120FDF7A1F935E00120FDF7DFF931E062
:105C80000120FDF7C5F92DE00120FDF703FA29E019
:105C90000120FDF7E9F925E078692A4BB0FA80F098
:105CA000FF26012140091E604FF03208FDF77CFA03
:105CB0001BE07B6933B1234BFF22012100201A60D6
:105CC000FDF772FA0120FDF731FA0BE07B6933B181
:105CD0001C4BFF22012100201A60FDF765FA01200C
:105CE000FDF736FA4FF03208FF260224FFF70AB913
:105CF0001548FEF73BFEFFF7BEB84FF0000904243D
:105D00002CE74FF03208FF260424FFF7FBB84FF0D2
:105D10003208FF260024FFF7F5B800BF1BB70008C4
:105D2000E7B10008081300202FB70008580C002026
:105D3000700C00206C0C00202C0C0020680C002043
:105D400068020020600200203CB70008F0B5234B39
:105D500087B01C680546002C3DD0214B984239D9AC
:105D600018226946BF20FDF7EFFBA0B11D480DF1D9
:105D7000010200233C2712F8011C567819501178B3
:105D80001C1807FB01610833402B616002F103021C
:105D9000F1D1012400E00446134B9D421BD9182287
:105DA000694640F2D710FDF7CFFBA0B10F480DF1C7
:105DB000010200233C2712F8011C56781950117873
:105DC0001D1807FB01610833402B696002F10302D3
:105DD000F1D100E00024204607B0F0BD38060020D5
:105DE000FF060100B4130020FF040200F41300209A
:105DF00070B5204B86B01B680BB9002038E00DF160
:105E0000010422461C4E00233C209D59991902F89A
:105E1000015C4D680833B5FBF0F1117000FB1151C6
:105E2000402B517002F10302EFD118226946BF20C6
:105E3000FDF7A2FB0028E0D0104D00233C2158596B
:105E40005A1904F8010C50680833B0FBF1F22270C3
:105E500001FB1202402B627004F10304EFD11822FF
:105E6000694640F2D710FDF787FB003018BF0120CC
:105E700006B070BD38060020B4130020F4130020D3
:105E800070B560B32D4E0025AC59A81914F0800FE1
:105E900021D0406898421ED104F0400011B1B0FA00
:105EA00080F04009B8B1C4F3C20004F00704A04276
:105EB00008D8904204D8944234BF0020012009E061
:105EC000002007E0944204D290428CBF00200120C1
:105ED00000E0012080BB0835402DD5D12AE0184EC6
:105EE0008559841915F0800F21D06468A3421ED112
:105EF00005F0400411B1B4FA84F46409BCB1C5F3EF
:105F0000C20405F00705AC4208D8A24204D3AA4255
:105F10008CBF0024012409E0002407E0AA4204D930
:105F2000A24234BF0024012400E0012424B9083037
:105F30004028D5D1002070BD012070BDF413002091
:105F4000B41300207047000070B50024254664207B
:105F5000FAF7B0FC002220211C4801F0D1FF4FF4D9
:105F60000C70FAF7A7FC01222021184801F0C8FFA5
:105F7000174E1420FAF79EFC3C233360202113486F
:105F800001F0B8FF10B925B9356802E00DB104B9C8
:105F900034683368002BF1D125B124B12C1B04EBFC
:105FA000840400E02C463220FAF784FC20210748C4
:105FB00001F0A0FF05467820FAF77CFC1E2C03D9DF
:105FC0006B1E5842584170BD002070BD000C01404E
:105FD0001C12002010B50E4C00222021204601F09A
:105FE0008FFF0520FAF766FC01222021204601F0F0
:105FF00087FF0A20FAF75EFC2021204601F07AFF95
:1060000004463220FAF756FC631E5842584110BD30
:10601000000C014070B5082601240025FFF7DAFFC7
:1060200000B125436400013EE4B2F7D1284670BDBB
:1060300038B504464518AC4204D0FFF7EBFF04F82E
:10604000010BF8E738BD000070B5064608250124AD
:1060500016EA04020ED000222021104801F050FF61
:106060000520FAF727FC0D480122202101F048FF06
:1060700050200CE02021094801F042FF5020FAF79F
:1060800019FC06480122202101F03AFF0520FAF709
:1060900011FC6400013DE4B2DAD170BD000C014096
:1060A00038B504464518AC4204D014F8010BFFF78C
:1060B000CBFFF8E738BD10B50446FFF745FF50B1F8
:1060C0003320FFF7C1FF08212046FFF7B1FFFFF79C
:1060D0003BFF012010BD2060606010BD37B5114D41
:1060E0002B68EBB90520FAF70DFC012401A82C6000
:1060F00001F0F8FE2146202002F088F81423202524
:106100008DF8073001A903230748ADF804508DF836
:10611000063001F099FE22462946034801F0F0FEC0
:1061200003B030BD780C0020000C014007B501A879
:1061300001F0D8FE0121082002F068F80123ADF833
:106140000430022301A98DF80630074810238DF88A
:10615000073001F079FE0548FEF75CFB0448FEF7C6
:1061600059FB03B05DF804FB000C014061B7000867
:10617000E7B1000810B5094C2368012B0CD00122AF
:106180001146074801F0BCFE0648FEF743FB0648EF
:10619000FEF740FB0123236010BD00BF6402002016
:1061A000000C014075B70008E7B1000810B5084CB5
:1061B000236863B100220121064801F0A1FE0648D0
:1061C000FEF728FB0548FEF725FB0023236010BDE2
:1061D00064020020000C014088B70008E7B1000805
:1061E000F0B50E4C002306258B4214D005FB03F2BC
:1061F0000778165DB7420CD12244B0F80170B2F8AE
:106200000160B74205D1B0F80360B2F803209642AE
:1062100002D00133E8E7FF231846F0BD800C0020D0
:1062200007B56846FDF71CFFB0B10D4A136801338E
:1062300013600C4A9DF805301068114620B9D80744
:1062400002D50123136007E003F001030B606846E9
:106250001421FFF7C5FF00E0FF2003B05DF804FB49
:10626000F80C00207C0C002073B5304E304C00251B
:1062700001212046FCF74CFC2046FEF7CBFA2D48C6
:10628000FEF7C8FA6846FDF7EBFE3046FDF7E8FE7C
:106290000028FAD07379DB07F7D43DB129463046A0
:1062A000FFF79EFFFF2801D00028EED10135142D05
:1062B00034D0AB1E112B2ED8DFE803F0090B0D0FE5
:1062C00011131517191B1D1F21232527292B1A4CC4
:1062D00022E01A4C20E01A4C1EE01A4C1CE01A4C2A
:1062E0001AE01A4C18E01A4C16E01A4C14E01A4C3A
:1062F00012E01A4C10E01A4C0EE01A4C0CE01A4C4A
:106300000AE01A4C08E01A4C06E01A4C04E01A4C59
:1063100002E01A4C00E01A4C0636A9E701211948A0
:10632000FCF7F6FB012002B070BD00BF800C00201E
:106330003AB90008E7B10008C6B70008DDB70008A1
:10634000F4B700080DB8000826B8000835B80008F2
:1063500044B8000855B8000866B800087FB80008BF
:1063600098B80008B3B80008CEB80008E8B800082C
:1063700002B900081EB90008ACB700089CB70008B5
:10638000C3B7000847B9000837B5134B186808B3FE
:10639000124D002404EB8400052269460430FDF709
:1063A000D3F8062363439DF800209DF802105A5548
:1063B0009DF801202B4442EA0122A3F801209DF818
:1063C00004109DF80320013442EA0122142CA3F8A2
:1063D0000320DFD103B030BD38060020800C002040
:1063E00073B5134B186800B3124D0024062606FB44
:1063F00004F35A5D2B448DF80020B3F8012004EB20
:1064000084008DF80120120A8DF80220B3F80330C1
:1064100005228DF8033069461B0A043001348DF8DB
:106420000430FDF7A9F8142CE1D102B070BD00BF13
:1064300038060020800C002007B50B46009201466C
:106440000022D020FDF7F8FCB0FA80F0400903B03C
:106450005DF804FB07B50B46009201460022D020F0
:10646000FDF74EFDB0FA80F0400903B05DF804FB83
:1064700037B5FDF7ABFC01220DF107013F20FFF717
:10648000DBFF012205460DF1070138B30720FFF7B6
:10649000D3FF08B9002435E09DF8073043B100234D
:1064A00001220DF1070107208DF80730FFF7D2FF19
:1064B00001220DF107010020FFF7BEFF044600286E
:1064C000E8D09DF807301A0619D503F07F038DF840
:1064D000073001220DF1070100200EE00E20FFF72A
:1064E000ABFF04460028D5D09DF807303BB18DF8AE
:1064F000075001220DF107010E20FFF7ABFF034B00
:1065000001221A60204603B030BD00BF680200209F
:1065100007B5254B1B68002B42D002680A2392FB6B
:10652000F3F103FB112202EB01128DF80020426807
:1065300092FBF3F103FB112202EB01128DF8012013
:10654000826892FBF3F103FB112202EB01128DF83A
:106550000220826901328DF80320C26892FBF3F1B8
:1065600003FB112202EB01128DF8042002690132B3
:1065700092FBF3F103FB112202EB01128DF80520CF
:1065800042690020643A92FBF3F103FB11230722D6
:1065900003EB011369468DF80630FFF75BFF00E05F
:1065A000184603B05DF804FB6802002013B5224BC7
:1065B0000446186800283CD0072269460020FFF7EF
:1065C0003BFFB0B39DF800200A23110902F00F022F
:1065D00003FB012222609DF80120110902F00F0245
:1065E00003FB012262609DF80220110902F00F02F4
:1065F00003FB0122A2609DF80320013AA2619DF8ED
:106600000420110902F00F0203FB0122E2609DF851
:106610000520110902F00F0203FB01229DF806106C
:10662000013A22610A0901F00F0103FB02136433EE
:10663000636102B010BD00BF6802002007B5104BB7
:106640001B68CBB10F4B98420DD901220DF1070108
:10665000DE20FCF779FF9DF807300A2B07D90023CD
:106660008DF8073003E000238DF8073001209DF8F6
:106670000720054B5A6000E0184603B05DF804FBA4
:1066800038060020FF0002006802002007B5094B11
:106690005B688DF80730084B186840B101220DF196
:1066A0000701DE20FCF768FF003018BF012003B0AF
:1066B0005DF804FB680200203806002010B5034C8A
:1066C0006060FFF7E3FF606810BD00BF6802002054
:1066D00013B50C4C236883B1022201A91120FFF7E6
:1066E000ABFE58B19DF805009DF80430C0F34000A2
:1066F00040EA43006368C01A00E0FF20A06002B0D7
:1067000010BD00BF68020020FCF720BE1FB503AA21
:1067100002A901A8FCF742FE48B1029B064A1BB938
:106720001068039B181A00E0FF20506000E0FF2073
:1067300005B05DF804FB00BF7402002007B5104BE4
:106740001B68CBB10F4B98420DD901220DF1070107
:10675000DF20FCF7F9FE9DF807300A2B07D900234C
:106760008DF8073003E000238DF8073001209DF8F5
:106770000720054B1A6000E0184603B05DF804FBE3
:1067800038060020FF0002007402002007B5094B04
:106790001B688DF80730084B186840B101220DF1D5
:1067A0000701DF20FCF7E8FE003018BF012003B02E
:1067B0005DF804FB740200203806002010B5034C7D
:1067C0002060FFF7E3FF206810BD00BF74020020C7
:1067D0000920FCF727BE00002DE9F843194E0746B3
:1067E000B146DFF86C800024B3682344092B04DD34
:1067F0000134042CF8D1BDE8F883002599E80A009B
:1068000003EB810308EB83031B5D2B41DB0714D5EE
:10681000F26853190A2B10DCB3680B20234400FBE9
:10682000032028442FB1084B01EB410100221944F9
:1068300001E03A460549FAF777FB0135042DDDD131
:10684000D6E700BF34140020FC0C0020110D0020FE
:1068500069B9000809280BD84B1C0B2B08D8054B2D
:106860000B2202FB0030405C003018BF0120704753
:1068700000207047140D00202DE9F74F0F46914678
:10688000164B00261C684FF0010A00EB8400C1EB98
:106890008004134801F1040B04443D460AFA06F350
:1068A00006EB0908625D1A420BD0092D01930CDC3E
:1068B000B8F10A0F09D841462846FFF7CBFF019BE4
:1068C00018B901355D45EDD101E0002003E0013646
:1068D000042EE2D1012003B0BDE8F08F3414002073
:1068E00069B9000838B5094CA568E2680135294640
:1068F0006068FFF7C1FF38B10020FFF76DFF01208E
:10690000A560FFF769FF012038BD00BF34140020E7
:106910002DE9F04FAB4EAC4D93B00024AB490123B1
:106920002144F26809A8FBF78FF9A94B9DF82420B0
:106930009DF8251033F8122033F8111062552A19EA
:1069400051709DF82610033433F81130152C9370D4
:10695000E4D19C4A0123D2689E4909A8FBF774F947
:106960009D4B00241C705C709C70204600229A494C
:106970000134FAF7D9FA6E2CF7D100231A4697485A
:10698000C118C2500B336E2B4A604FF00005C1F89E
:106990000720F5D1924F07233A68924CB2FBF3F3EC
:1069A000914EC3EBC303D31A84E82800F35C0120A3
:1069B000C3F10202A260C3F10B03022293FBF2F3C4
:1069C000E360FFF709FF3223029301954FF0010ABC
:1069D00005970696FAF7A4FA844E0027FCF776FF8F
:1069E00009280DD196F84C30472B09D196F84D3037
:1069F000542B05D17D4B93F84E30712B08D12DE1EE
:106A00000A20F9F767FF029B0137BB42E6D140E05D
:106A10006D2B35D007D8642B2FD06C2B39D1714F0B
:106A2000FE68013E07E0722B02D0752B0FD030E0DC
:106A30006C4FFE6801363246B9687868FFF71CFF74
:106A40000028C7D00020FFF7C7FEFE6011E0654BAD
:106A50005E68DA68032E14BF013600269968304656
:106A6000FFF70AFF0028B5D00020FFF7B5FE5D4B09
:106A70005E600120FFF7B0FEACE7FFF733FFA9E748
:106A8000FFF730FF28B1FAF74BFA3220F9F722FF6F
:106A9000F6E7FFF727FF00289CD12268E368A76884
:106AA0000393531CDBB2049363684FF0010C03EBB8
:106AB00082034F4A02EB830B0B2202FB07F907927A
:106AC000039B0CFA00FE1E18444B06EB0901194407
:106AD00000231BF8038018EA0E0F0DD007EB030804
:106AE000B8F1090F08D80A2E9FBF079A02FB03F8D6
:106AF0009DF8102001F808200133042BE9D1013062
:106B00000428DDD14FF000094FF00908002739466D
:106B10004046FFF79FFE00283DD001370B2FF6D1EE
:106B2000464607FB08F73EB32C4BA7F10C0B5B4422
:106B300003934FF0000B039B594613F8012F304687
:106B4000DA7203930492FFF785FE38B1049A1E4B64
:106B5000013A02EB42011944002201E002461E49BB
:106B60000BEB07000BF1010BFAF7DEF9BBF10B0F92
:106B7000E1D1013E0B3FD6E73746184B3046F7547C
:106B8000002215490136FAF7CFF90B2EF5D109F19C
:106B9000010908F1010818F1FF38B7D2B9F1000F67
:106BA0003CD0B9F1020F07D0B9F1030F06D0B9F10B
:106BB000010F1FD128231FE064231DE04FF49673BB
:106BC0001AE000BF30000020FC0C002054B900087F
:106BD000D4A40008D9B90008110D0020140D00201C
:106BE000280C0020341400207C0200202C120020ED
:106BF00069B900084FF4966303FB0A55019B4B44A7
:106C0000092B019308D9029B0AF1010A092B84BFC1
:106C1000053B029300230193FAF782F9059B0120BB
:106C20001A680723B2FBF3F3C3EBC303D31A0022A2
:106C30006260069A2360D35CC3F10202A260C3F1D2
:106C40000B03022293FBF2F3E360FFF7C5FD201D67
:106C500007C8FFF711FE00287FF4BCAEC820F9F783
:106C600039FE2A4605490AA801F0E0FF01210AA8D9
:106C7000FBF74EFF13B0BDE8F08F00BFDCB9000892
:106C800007B50E4B5B69002BB8BF5B428DF8053032
:106C90000B4BA8BF2B221868B6BF2D228DF80420FD
:106CA0008DF8042038B1022201A9BA20FCF764FC57
:106CB000003018BF012003B05DF804FB84020020FF
:106CC0003806002013B5134B134C1B68ABB11022D0
:106CD0002146AA20FCF738FC78B1022201A9BA208B
:106CE000FCF732FC48B19DF804209DF805302D2AB0
:106CF00063610BD15B42636108E0102207490648DB
:106D000001F0ECFF01236361002000E0012002B0EC
:106D100010BD00BF3806002084020020E8B900083A
:106D200008B5084B1B685BB110220749AA20FCF785
:106D300023FC28B1FFF7A4FF003018BF012008BDD5
:106D4000002008BD380600208402002010B504464B
:106D500001460948FDF7FAFD04F10C03182B07D88A
:106D6000064B5A69944205D05C61FFF789FF01E048
:106D7000002010BD012010BDF7B9000884020020DA
:106D800008B50146074801F084FF074B186838B181
:106D900010220449AA20FCF7EFFB003018BF0120A5
:106DA00008BD00BF840200203806002000B5084A54
:106DB00089B013782BB1074901A801F037FF01A86A
:106DC00000E00548FCF782FE09B05DF804FB00BF57
:106DD000840200200ABA000814BA000873B5264BD2
:106DE000264A5B690A444FF4616101FB032302AE4A
:106DF00046F8043D0546304601F008FD03690446A7
:106E0000DA1E052A2FD9022B09D18269C3689B1A81
:106E1000182B0FDD3ABB8368012B24DC0AE0092B19
:106E200008D18269C3689B1A182B1CDD12B98368CC
:106E3000022B18DD63696B6123692B61E368EB60EA
:106E40006269216902F26C720131E068F9F73AFA7D
:106E5000A861236A2B62A368AB6063686B602368D8
:106E60002B6002B070BD019B304603F56163019356
:106E700001F0CCFC0446DDE7840200208081557CD3
:106E800010B504460D48FCF735FC2046FCF732FCF3
:106E90000B48FCF72FFCFCF75FFCFCF717FD032801
:106EA0000146FAD00028F8D0012806D00548FDF7A1
:106EB0004DFDBDE81040FDF7D7BC10BD19BA000864
:106EC000E7B100081EBA000800B58A788BB00B78CD
:106ED00001924A7805490092024602A801F0A6FEF6
:106EE00002A8FFF7CDFF0BB05DF804FB4ABA00081B
:106EF00000B593B00B4600920549024602A801F086
:106F000095FE02A8FFF7BCFF13B05DF804FB00BFBD
:106F10005FBA000800B58BB00B46009205490246E7
:106F200002A801F083FE02A8FFF7AAFF0BB05DF8EC
:106F300004FB00BF68BA000800B5C1F307238BB09B
:106F40000246009302A8CBB2044901F06FFE02A8EA
:106F5000FFF796FF0BB05DF804FB00BF73BA0008A3
:106F600000B591B00B4602460449684601F05EFE4A
:106F70006846FFF785FF11B05DF804FB81BA000891
:106F800000210846FFF7D8BF024B0320996AFFF79C
:106F9000D3BF00BF30000020024B04201968FFF768
:106FA000CBBF00BF30000020024B0620D968FFF79E
:106FB000C3BF00BF30000020024B08205969FFF713
:106FC000BBBF00BF30000020024B0A20D969FFF789
:106FD000B3BF00BF30000020024B0B205968FFF701
:106FE000ABBF00BF30000020024B0E201969FFF735
:106FF000A3BF00BF30000020024B0F209968FFF7AD
:107000009BBF00BF30000020024B10205988FFF7C3
:1070100093BF00BF7C090020024B11209988FFF725
:107020008BBF00BF7C090020024B1220D988FFF7DC
:1070300083BF00BF7C090020024B15209968FFF731
:107040007BBF00BF68020020024B17205968FFF782
:1070500073BF00BF7402002001490120FFF780BF09
:1070600023B4000801490220FFF77ABF081300206B
:1070700001490420FFF774BF840200200149052064
:10708000FFF76EBF4414002001490620FFF768BFD8
:107090006514002001490720FFF762BF8614002015
:1070A00001490820FFF75CBF8F14002000B50C4B8E
:1070B0008FB09A680B490492DA6806A803921A699D
:1070C00002925A6901929A690092DB69002201F0EA
:1070D000ADFD06A8FFF7D4FE0FB05DF804FB00BFBE
:1070E0000813002089BA000830B5094D91B000247A
:1070F00055F824303BB122460649684601F096FD1A
:107100006846FFF7BDFE0134082CF1D111B030BD47
:1071100028020020A7BA000801490020FFF7D4BECA
:107120007800002001490120FFF7CEBE7B0000203F
:1071300038B50E4D00242A6D21460D48FFF7D8FEC4
:10714000AA6D21460B48FFF7E5FEEA6D21460A4885
:10715000FFF7E0FE2A6E214608480134FFF7DAFE09
:107160000C2C05F11405E6D138BD00BF300000201D
:10717000B0BA0008B3BA0008B6BA0008B9BA000835
:1071800038B5104D0024D5F8402121460E48FFF7B0
:10719000AFFED5F8442121460C48FFF7BBFED5F8D9
:1071A000482121460A48FFF7B5FED5F84C21214673
:1071B00008480134FFF7AEFE022C05F11005E2D1BC
:1071C00038BD00BF30000020BCBA0008BFBA0008BC
:1071D000C2BA0008C5BA000838B5104D0024D5F869
:1071E000602121460E48FFF783FED5F86421214631
:1071F0000C48FFF78FFED5F8682121460A48FFF7B3
:1072000089FED5F86C21214608480134FFF782FE3B
:10721000042C05F11005E2D138BD00BF300000207C
:10722000C8BA0008CBBA0008CEBA0008D1BA000824
:1072300030B58BB0FFF7A4FE6D4B01201968FFF746
:107240007BFE6C4B6C4DD9886C4C1D20FFF774FE97
:1072500029680220FFF770FEFFF796FEE16A1E2004
:10726000FFF76AFEFFF798FE08210520FFF764FE8E
:10727000FFF79AFEA1690720FFF75EFEFFF79CFE6D
:1072800094F838100920FFF757FE94F834101920AD
:10729000FFF752FE94F835101A20FFF74DFE94F8D0
:1072A00036101B20FFF748FE94F837101C20FFF71C
:1072B00043FEFFF789FEFFF78FFE616C0C20FFF79E
:1072C0003BFE216C0D20FFF737FEFFF78DFEFFF729
:1072D00093FEFFF799FEFFF79FFEFFF7A5FE484BD1
:1072E000132059690029BDBF494289B241F4807118
:1072F00089B2FFF721FE434B14201968FFF71CFEEB
:10730000FFF79AFE69681620FFF716FEFFF79CFE4E
:107310003D4B18201968FFF70FFED4F8E0111F202D
:10732000FFF70AFEFFF798FEFFF79CFEFFF7A0FEAF
:10733000FFF7A4FEFFF7A8FEFFF7ACFEFFF7B0FED5
:1073400032490920FFF70CFE31490A20FFF708FEF9
:10735000FFF7ACFEFFF7C8FEFFF7DEFEFFF7E2FE29
:10736000FFF7E6FEFFF70CFFFFF736FF294D00247D
:1073700005EBC4035B6855F8342027490192C3F339
:1073800007220092DBB2224602A801F04FFC013432
:1073900002A8FFF775FD082CEAD1204D002405EB6B
:1073A000C4035B6855F834201D490192C3F30722DA
:1073B0000092DBB2224602A801F038FC013402A898
:1073C000FFF75EFD082CEAD1164D002455F8043F66
:1073D000002200931449234602A801F027FC01343F
:1073E00002A8FFF74DFD402CF0D10BB030BD00BF1F
:1073F000380600200813002068020020300000201A
:107400008402002020120020740200203413002087
:1074100074130020B4130020D4BA0008F413002021
:10742000E6BA0008CC010020F8BA000838B51D4BB8
:107430001B680BB9002038BD1B4C2022214640F2AE
:107440004710FCF781F825460028F3D0202204F1EC
:10745000210140F26710FCF777F80028EAD00822F3
:1074600004F1420140F28710FCF76EF80028E1D0E9
:10747000082204F14B0140F28F10FCF765F8002858
:10748000D8D094F84230303B092B04D894F84B30D4
:10749000303B092B04D9002385F8423085F84B3066
:1074A000012038BD380600204414002010B52022E9
:1074B000134940F24710FCF75FF8A0B1114C236864
:1074C0008BB12022104940F26710FCF755F850B1FB
:1074D000236843B108220D4940F28710FCF74CF8AD
:1074E00008B123680BB9002010BD0822084940F2FA
:1074F0008F10FCF741F80028F5D0012010BD00BF27
:107500004414002038060020651400208614002052
:107510008F14002010B5074C01462022204601F0B0
:10752000DDFB2146BDE81040202240F24710FCF769
:1075300023B800BF4414002008B5014620220748A4
:1075400001F0CCFB064B1B683BB1BDE80840202294
:10755000024940F26710FCF70FB808BD651400201F
:107560003806002010B504462E222C21F8F7F7FE2D
:1075700008222146074801F0B1FB074B1B683BB1CD
:10758000BDE810400822034940F28710FBF7F4BF22
:1075900010BD00BF861400203806002010B5044638
:1075A0002E222C21F8F7DBFE08222146074801F0A5
:1075B00095FB074B1B683BB1BDE81040082203490F
:1075C00040F28F10FBF7D8BF10BD00BF8F14002012
:1075D0003806002010B51F4C98B022782346BAB365
:1075E00094F84220D2B194F84B20BAB11A496846B7
:1075F00001F04FFB2146684601F03CFB1749684605
:1076000001F038FB04F14201684601F033FB1349F5
:10761000684601F02FFB04F14B010FE093F8213095
:10762000B3B10D49684601F034FB0A49684601F0E0
:1076300021FB0A49684601F01DFB0949684601F033
:1076400019FB0849684601F015FB6846FCF73EFA4D
:1076500018B010BD4414002006BB000810BB000881
:10766000651400200EBB000807B501A800F03AFC25
:107670000121042000F0CAFD8023ADF8043001A9E7
:10768000482304488DF8073000F0DEFB03B05DF8B6
:1076900004FB00BF0008014008B58021034800F04A
:1076A00029FCB0FA80F0400908BD00BF0008014085
:1076B000F0B5394B394DA3F11802002814BF184614
:1076C0001046374C374B2E6822681B689A4245D2C9
:1076D00040F20A27344B1968344B226807FB013308
:1076E00002EB42021344024600F10801802793F89E
:1076F00001E001321EEA070F14BF4FF0390E4FF0C0
:10770000210E02F801EC8A424FEA5707EFD100F14F
:107710001002802793F800E001311EEA070F14BF22
:107720004FF0390E4FF0210E01F801EC8A424FEA7A
:107730005707EFD1183080219F7801320F4214BFD4
:107740003927212702F8017C82424FEA5101F3D107
:10775000236806F11801013323601AE03146DFF88F
:1077600050E018234FF0000CDEF800708C1B8F42A5
:1077700000EB040206D9013B00F804C001F101014D
:10778000F2D106E013440020934202D0107001327F
:10779000FAE72960F0BD00BFC8110020880D002065
:1077A000900D0020940D0020840D00209C0D0020E1
:1077B000E011002008B5402000F02EFB28B1402049
:1077C00000F038FB0020FFF773FF202000F024FBBF
:1077D000A0B1202000F02EFB094B1A68094B1B6852
:1077E0009A4204D2BDE808400120FFF761BF0021A2
:1077F000054800F0FCFA054B00221A6008BD00BFE6
:10780000880D0020E01100201C0002408C0D00209B
:10781000F8B5AE28284B28BFAE201C68002CFCD140
:10782000264D274E2B68274A3360B3FA83F35B0952
:107830002B60254B01271C60244B1C6018234343FD
:10784000ED331360224B18602046FFF731FF012013
:10785000FFF72EFF184B21461E481F6000F09BFDCE
:1078600021461D4800F0C3FA30211B4800F0D2FA2F
:107870003A460621184800F0C5FA3946164800F085
:10788000B6FA394640F20A27124800F084FD13493F
:10789000336804EB440007FB03032A680B4407FB2F
:1078A00002021888013488529B7801EB020EAE2C3C
:1078B0008EF80230ECD1F8BD8C0D0020980D002020
:1078C000840D0020E0110020880D0020900D002084
:1078D000940D0020002C01401C0002409C0D002053
:1078E000AD2830B50FD840F20A25074B00EB400019
:1078F0001B680C7805FB0300044A145413184A78DB
:107900005A708A789A7030BD980D00209C0D002026
:10791000F0B540F20A24104BAE291D680F4E04FB4F
:1079200005F528BFAE2100238B420DD090F800E072
:1079300003EB43042C4406F804E037194478013380
:107940007C708478BC70EFE722B1BDE8F040184647
:10795000FFF75EBFF0BD00BF980D00209C0D00201A
:1079600030B55C4B95B0002268461A6000F0BAFA58
:107970000121042000F04AFC282369464FF480745A
:107980008DF80330544803238DF80230ADF80040E1
:1079900000F05AFA0120F8F79DFF21464E4800F00A
:1079A000A9FA012807D14D48FCF734FF4C48FCF7F1
:1079B00031FF1C2306E04B48FCF72CFF4848FCF73E
:1079C00029FF18238DF803306946032342488DF8B8
:1079D000023000F039FA00224FF480713E4800F086
:1079E0008FFA02A800F0C4FC05A800F0CAFC01212F
:1079F0004FF4006000F00AFC01210846002400F06A
:107A0000F9FB5A2302A938480125ADF80C30ADF82E
:107A10000840ADF80E40ADF80A4000F01BFC6023B2
:107A200005A93148ADF81430ADF81650ADF81A403C
:107A3000ADF81C4000F058FC08212B4800F0DCFC9D
:107A40002946294800F0CCFC2946274800F0AFFC25
:107A50002A464FF40071244800F0B7FC0C2301A81B
:107A60008DF804308DF805408DF806408DF80750EC
:107A700000F042F809A800F0ADF921461B4800F0DB
:107A8000B6F91A4800F010F920231193184B09A9F0
:107A900009934FF480730F9330230C9380230E933C
:107AA0004FF44053129310230B93124B0F480A9339
:107AB00010940D94139400F06FF92A46AE2109A892
:107AC0008DF824408DF825408DF82640FFF720FFE3
:107AD00015B030BD8C0D00200008014014BB00081B
:107AE000E7B1000835BB0008002C01401C00024033
:107AF000342C0140B0110020C27810B503780AB3CD
:107B0000164A03F16043D1684278C943C1F30221A8
:107B1000C1F1040402FA04F40F22CA40817803F58B
:107B200061430A4022431201D2B283F80023037852
:107B30000122590903F01F0302FA03F3084A42F82D
:107B4000213010BD5A09012103F01F0301FA03F38C
:107B50000349203241F8223010BD00BF00ED00E0A3
:107B600000E100E0436810B523F470220B6822F4B2
:107B7000807213430A7943EA022343608B68CA6820
:107B800084681A43084B234013434A7943EA42036B
:107B90008360C36A23F470020B7C013BDBB242EAD0
:107BA0000353C36210BD00BFFDF7F1FF0023036064
:107BB000037143718360C36001230374704783685A
:107BC00011B143F0010301E023F00103836070472A
:107BD000836843F00803836070478068C0F3C00087
:107BE0007047836843F00403836070478068C0F384
:107BF00080007047836811B143F4A00301E023F4CF
:107C0000A00383607047092970B50DD9A1F10A045A
:107C1000C66804EB44040725A54026EA050503FAD7
:107C200004F42C43C4600AE0066901EB4104072513
:107C3000A54026EA050503FA04F42C430461062A4C
:107C40000CD8013A446B02EB82021F23934024EAD2
:107C5000030301FA02F21A43426370BD0C2A0CD8E6
:107C6000073A046B02EB82021F23934024EA0303CA
:107C700001FA02F21A43026370BD0D3AC46A02EBC4
:107C800082021F23934024EA030301FA02F21A43FB
:107C9000C26270BDC06C80B270470368194214BFE5
:107CA00001200020704700004FF6FE730268134069
:107CB00003600023036043608360C360284B9842E5
:107CC00001D1284A27E0284B984201D1254A2AE0D1
:107CD000264B984201D1234A2DE0254B984201D1F1
:107CE000204A30E0234B984201D11E4A33E0224B18
:107CF000984204D11B4A536843F470032EE01F4B93
:107D0000984204D1174A536843F0706326E01C4B35
:107D1000984204D11B4A536843F00F031EE01A4BEC
:107D2000984204D1174A536843F0F00316E0174B0A
:107D3000984204D1134A536843F470630EE0144B25
:107D4000984204D10F4A536843F4704306E0114B44
:107D5000984204D10B4A536843F470235360704730
:107D600008000240000002401C00024030000240B7
:107D700044000240580002406C0002408000024073
:107D800008040240000402401C0402403004024087
:107D900044040240580402400A6A10B58C68036823
:107DA00014430A6923F4FF4314434A6923F0700320
:107DB00014438A691443CA6914434A6A14438A6A99
:107DC000224313430360CB6843600B6883604B68B6
:107DD000C36010BD0023036043608360C360036120
:107DE00043618361C361036243628362704719B177
:107DF000036843F0010303E04FF6FE73026813408B
:107E00000360704703680AB1194301E023EA0101E6
:107E10000160704741607047C3004CBF034B044B87
:107E20001B68034214BF0120002070470004024079
:107E300000000240C3004CBF014B024B586070472A
:107E40000004024000000240CA78F0B502F00F03BF
:107E5000D20644BF8A7813430A78F2B1026800243C
:107E600001274FF00F0E0D8807FA04F636EA0505D4
:107E70000FD1A5000EFA05FC22EA0C0203FA05F563
:107E80002A43CD78282D01D1466102E0482D08BF54
:107E900006610134082CE6D102600A88FF2A20D945
:107EA0004268002401274FF00F0E04F108050E88E8
:107EB00007FA05F535EA06060FD1A6000EFA06FC0C
:107EC00022EA0C0203FA06F63243CE78282E08BFC7
:107ED0004561CE78482E08BF05610134082CE4D1F5
:107EE0004260F0BD4FF6FF730380022383700423CA
:107EF000C37070478368194214BF01200020704787
:107F00000AB10161704741617047000030B5002837
:107F1000154A00F44015B4BFD3695368B5F5401F46
:107F200084B206D1556823F0706325F07065556002
:107F30000EE0C20255BF420D03221201C0F30345F9
:107F40004CBFAA4004FA02F223EA020343F0706332
:107F500019B1420D120194402343034A0028B4BFD3
:107F6000D361536030BD00BF0000014008B50B4B2A
:107F70000121984207D14FF4001000F05FF9002171
:107F80004FF4001006E04FF4800000F057F9002194
:107F90004FF48000BDE8084000F050B900540040A4
:107FA00070B586B00446868801A80D4600F0DEF85C
:107FB000039A2E4826F03F06B2FBF0F03604360C4A
:107FC00081B20E43A6802388294E23F001031B04AF
:107FD0001B0C23802B68B3420AD85B00B2FBF3F37F
:107FE00001319BB2032B89B298BF0423218423E083
:107FF0004BF6FF71EE888E421BBF19214B4303EBFA
:108000004303B2FBF3F30BBFB2FBF3F39BB29BB2A0
:1080100043F48043C3F30B020AB943F001034FF466
:10802000967101FB00F24FF47A7192FBF1F201328A
:1080300092B243F400432284A38323889BB243F08B
:10804000010323802388A98823F481636A8923F0AC
:1080500002031B040A431B0C13439BB22380AA890F
:108060002B8913439BB2238106B070BD40420F00A1
:10807000A086010041F288334BF6FF7203600023B3
:108080008380038143814FF48043C28083817047A2
:10809000038819B19BB243F0010303E023F001030D
:1080A0001B041B0C03807047038819B19BB243F477
:1080B000807303E023F480731B041B0C0380704760
:1080C000038819B19BB243F4007303E023F40073F7
:1080D0001B041B0C03807047038819B19BB243F447
:1080E000806303E023F480631B041B0C0380704750
:1080F00001827047008AC0B2704712B141F001019D
:1081000001E001F0FE0189B201827047038829B1C4
:108110006FEA43436FEA53439BB201E0C3F30E039C
:108120000380704782B00023009301930B0F0190EE
:108130000093009B21F07F4113B1019B143302E0B7
:10814000019B090C18330193019B1B68194214BF52
:108150000120002002B07047034A536823F44043D3
:1081600018435060704700BF0010024010B51C4A11
:10817000536803F00C03042B01D0082B01D0194BDA
:108180000EE053685168C3F38343CC0303F1020349
:1081900002D55168890301D5134900E011494B43C9
:1081A00003605368114CC3F30313E15C0368CB40D5
:1081B00043605168C1F30221615C23FA01F18160DF
:1081C0005168C1F3C221615CCB40C3605268084969
:1081D000C2F381328A5CB3FBF2F3036110BD00BFCE
:1081E0000010024000127A0000093D00A0020020A9
:1081F0009C020020044B5A6909B1104301E022EAB5
:1082000000005861704700BF00100240044B9A699B
:1082100009B1104301E022EA00009861704700BFF5
:1082200000100240044BDA6909B1104301E022EA70
:108230000000D861704700BF00100240044B1A696B
:1082400009B1104301E022EA00001861704700BF45
:1082500000100240224A038890429BB212D002F5DD
:10826000006290420ED0B0F1804F0BD0A2F5983250
:10827000904207D002F58062904203D002F58062FE
:10828000904203D14A8823F070031343154A904269
:1082900008D002F5806290421FBF23F44073CA8861
:1082A0009BB2134303808B8883850B8803850C4B1B
:1082B00098420FD003F5006398420BD003F540635A
:1082C000984207D003F58063984203D003F580639A
:1082D000984201D10B7A038601238382704700BF45
:1082E000002C014000100040038C70B523F0010306
:1082F0001B041B0C0384028C8688038B0D8823F0DF
:1083000073031B041B0C1D4322F002020C894B88D3
:108310001204120C23431343144AB6B290429BB288
:108320000FD002F5006290420BD002F540629042FD
:1083300007D002F58062904203D002F5806290423D
:108340000ED14C8923F008031C438B8824F00404CD
:1083500026F4407223438E89CC893443224396B25B
:1083600086800583CA888286038470BD002C014004
:108370004FF6FF73838000230380C3804380037222
:1083800070470023038043808380C380038143813F
:108390008381C3817047038819B19BB243F0010305
:1083A00003E023F001031B041B0C03807047B0F8AB
:1083B000443029B16FEA43436FEA53439BB201E073
:1083C000C3F30E03A0F84430704783899BB20AB10F
:1083D000194301E023EA010181817047FFF7F5BFEE
:1083E000038819B19BB243F0800303E023F08003BC
:1083F0001B041B0C03807047038B23F008031B0432
:108400001B0C194301837047C94389B2018270472D
:1084100070B50E460446038ACA889BB223F44053C3
:108420001343038282898988338992B20B4371890D
:1084300022F4B0520B4322F00C0213439BB283810F
:10844000838AB2899BB223F4407386B0134383823C
:1084500001A8FFF78BFE174A039B049D31689442E5
:1084600018BF1D4619226A43A389642613F4004FDE
:1084700014BF4D008D00B2FBF5F5B5FBF6F0A289F7
:1084800000010109120406FB115307D5D90032314E
:10849000B1FBF6F202F00702104306E01A01323295
:1084A000B2FBF6F303F00F03184380B2208106B04D
:1084B00070BD00BF003801404FF4165303600C221A
:1084C00000238380C3800381428183817047838935
:1084D00019B19BB243F4005303E023F400531B048F
:1084E0001B0C83817047012310B5C1F342149C42D9
:1084F00001F01F0103FA01F101D10C3003E0022C5D
:108500000CBF1030143003680AB1194301E023EAAC
:108510000101016010BDC1F30801818070478088AE
:10852000C0F308007047838929B16FEA43436FEABB
:1085300053439BB201E0C3F30E03838170470123D1
:1085400010B5C1F3421401F01F029C4203FA02F27B
:1085500001D1838903E0022C0CBF038A838A9BB27A
:108560001340028892B243B10123090A03FA01F1D0
:108570000A4214BF1846002010BD184610BD090A53
:10858000012303FA01F1C94389B201807047000059
:108590000649074A074B9A42BEBF51F8040B42F8FE
:1085A000040BF8E70448804704480047C0BD0008B2
:1085B00000000020800300204986000849010008CF
:1085C0001F49204A002301E041F8043B9142FBD3BC
:1085D000FCF7C6FAFEE7FEE7FEE7FEE7FEE7FEE78A
:1085E000FEE7FEE7FEE7FEE7FEE7FEE7FEE7FEE763
:1085F000FEE7FEE7FEE7FEE7FEE7FEE7FEE7FEE753
:10860000FEE7FEE7FEE7FEE7FEE7FEE7FEE7FEE742
:10861000FEE7FEE7FEE7FEE7FEE7FEE7FEE7FEE732
:10862000FEE7FEE7FEE7FEE7FEE7FEE7FEE7FEE722
:10863000FEE7FEE7FEE7FEE7FEE7FEE7FEE7FEE712
:10864000800300209C140020384B82B01A6842F04E
:1086500001021A605968364A0A405A601A6822F0C4
:10866000847222F480321A601A6822F480221A601E
:108670005A6822F4FE025A604FF41F029A600022E8
:10868000009201921A6842F480321A601A6802F469
:1086900000320192009A01320092019A1AB9009AAE
:1086A000B2F5A06FF2D11A6812F4003218BF01229D
:1086B0000192019A012A05D01E4B4FF000629A6088
:1086C00002B070471C4A116841F010011160116836
:1086D00021F003011160116841F0020111605A6834
:1086E0005A605A685A605A6842F480625A605A68FE
:1086F00022F47C125A605A6842F4E8125A601A68EE
:1087000042F080721A601968084A8901FBD55168E5
:1087100021F003015160516841F0020151605A6833
:1087200002F00C02082AFAD1C6E700BF001002408E
:108730000000FFF800ED00E000200240114A124B5B
:10874000516801F00C01042901D0082901D00F491A
:108750000EE051685068C1F38341C00301F102018A
:1087600002D55068800301D5094800E0074841431D
:10877000196052680749C2F30312895C1A68CA403B
:108780001A60704700100240C002002000127A00F8
:1087900000093D00B002002008B5074B044613B1A4
:1087A0000021AFF30080054B1868836A03B1984736
:1087B000204601F0F9FD00BF000000005CBB00088E
:1087C0000E4B70B51E460E4C0025E41AA410A542AF
:1087D00004D056F8253098470135F8E701F0E6FD5A
:1087E000084B094C1E46E41AA4100025A54204D0EB
:1087F00056F8253098470135F8E770BD780300201A
:1088000078030020780300207C03002038B5074B54
:1088100005461C68E36B1BB9242000F0EFF8E06309
:10882000E16B2846BDE8384000F002B82403002080
:108830002DE9F0410C46804600F09AFD214607469E
:10884000404600F099FD4669044606F26C76B3078F
:1088500005D1642296FBF2F302FB13634BB94FF48C
:10886000C87596FBF5F305FB1365B5FA85F35B094F
:1088700000E001235F4A302505FB032500F072FB71
:1088800000F072FB5C4B1B68F3B17B689E4205D124
:108890003968D8F80030FA6941B90AE0304600F08A
:1088A000B9FA0028F4D14FF0FF330DE0934208DB12
:1088B00001E0934207DABA6B9342ACBF0023012375
:1088C00002E0002300E001232362236A3C20012B05
:1088D0000CBFF96B396A4FF4616391FBF3F603FB4C
:1088E000161393FBF0F200FB123061682368891ABB
:1088F000A2681B1A921B3B2B23606160A26003DD00
:10890000013161603C3B04E0002B03DA0139616016
:108910003C33236063683B2B03DD0132A2603C3BA8
:1089200004E0002B03DA013AA2603C336360A368E1
:10893000172B22DDE269183B0132E261A269A360D4
:108940000132062AC8BF0022A261E268236901320F
:10895000E26055F823108A4246DD01330C2B08BF34
:108960006369A2EB0102E26005BF013300222361CB
:10897000226104BF6361E26136E0002B34DAE26910
:108980001833013AE261A269A360013A48BF0622A6
:10899000A261E268013AE26032BB2369013B01D483
:1089A00023611DE00B23236163695A1E12F0030F3C
:1089B000626103F26B7305D1642193FBF1F201FB59
:1089C00012324AB94FF4C87193FBF1F201FB123332
:1089D000B3FA83F35B0900E0012303F5B673E361A7
:1089E000236955F82330E36000F0BDFA2046BDE866
:1089F000F08100BF60BB000808120020024B014656
:108A0000186800F06BB800BF24030020024B014639
:108A1000186800F017B800BF2403002010B5431EEB
:108A20000A44914204D011F8014B03F8014FF8E7D2
:108A300010BD03460244934202D003F8011BFAE73B
:108A40007047000038B50546002944D051F8043C71
:108A50000C1F002BB8BFE41800F024FD1E4A136859
:108A6000114613B96360146030E0A3420DD9226847
:108A7000A018834201BF18685B6812182260636007
:108A80000C6023E0A24203D813465A68002AF9D1A9
:108A900018681918A1420BD1216801445818824264
:108AA000196013D110685268014419605A600DE0D2
:108AB00002D90C232B6009E021686018824201BFB3
:108AC000106852680918216062605C602846BDE841
:108AD000384000F0E8BC38BDE811002070B5CD1C6E
:108AE00025F0030508350C2D38BF0C25002D064652
:108AF00001DBA94202D90C23336046E000F0D2FC2E
:108B0000234B1C681A462146A1B10B685B1B0ED48F
:108B10000B2B03D90B60CC18CD501EE08C420BBF41
:108B200063684B681360636018BF0C4615E00C4621
:108B30004968E9E7174C23681BB9304600F066F82E
:108B400020602946304600F061F8431C18D0C41C50
:108B500024F00304A0420DD12560304600F0A3FCB0
:108B600004F10B00231D20F00700C31A0ED05A4257
:108B7000E25070BD211A304600F048F80130EBD1C8
:108B80000C233360304600F08EFC002070BD00BF27
:108B9000E8110020E4110020194B10B51C68A36BEC
:108BA000D3B91820FFF72AFF43F20E33A0630380E6
:108BB0004AF6CD33438041F2342383804EF26D6315
:108BC000C3804DF6EC630381052343810B2383812E
:108BD00001220023C0E90423A16B0A4C0B694869F8
:108BE0005C43094A02FB0040A3FB02230132034419
:108BF00043F10003C1E9042323F0004010BD00BF8E
:108C0000240300202DF451582D7F954C38B5064C87
:108C1000002305460846236001F0B8FB431C02D13F
:108C2000236803B12B6038BD981400200EB400B542
:108C30004FF402719CB0ADF814106FF00041049134
:108C400007914FF6FF711DAB02900690084853F84C
:108C5000042BADF81610006802A9019300F07EFC09
:108C6000029B00221A701CB05DF804EB03B0704741
:108C700024030020024610B513461C780132002C54
:108C8000FAD1013B11F8012B03F8012F002AF9D189
:108C900010BD034611F8012B03F8012B002AF9D16E
:108CA0007047034613F8012B002AFBD1181A01382C
:108CB000704730B582B1451E013915F8013F11F8F2
:108CC000014FA34206D1EC431444E04201D0002BF3
:108CD000F3D11C46181B30BD104630BD034610B5FD
:108CE00042B111F8014B013A03F8014B002CF7D1C6
:108CF0001A4400E010BD934202D003F8014BFAE79A
:108D000010BD00002DE9F0470E4680463B48D0F8E4
:108D10000090354615F8014B09EB0400407800F04F
:108D2000080000F0FF0708B12E46F2E72D2C03D112
:108D3000B51C7478012703E02B2C04BF7478B51C94
:108D400013B1102B0AD153E0302C4FD1287800F00A
:108D5000DF00582845D16C78102302354FF0FF3CD6
:108D6000BCFBF3FC03FB0CFA00266FEA0A0A304650
:108D700009EB040E9EF801E01EF0040F01D0303C18
:108D80000BE01EF0030E1AD0BEF1010F0CBF4FF026
:108D9000370E4FF0570ECEEB0404A3420FDD002E2A
:108DA00008DB604506D801D1544503DC03FB0040D5
:108DB000012601E04FF0FF3615F8014BD8E7002EF1
:108DC00007DA2223C8F800304FF0FF302AB9BDE897
:108DD000F08707B1404272B106B1691E1160BDE86B
:108DE000F0873024002BB9D10823B7E70A23B5E771
:108DF000302CABD0B2E7BDE8F08700BF30030020D5
:108E000013460A46014602480068FFF77BBF00BFD1
:108E1000240300202DE9F74F044600F0A9FA40F2A0
:108E2000B1739C4240F3968040F26D156FF4F66387
:108E3000E318A4F2B2729B1005FB0235A4F26D7226
:108E40006FF0630392FBF3F36FF4C8622B44A51831
:108E50004FF4C87294FBF2F795FBF2F502FB17474B
:108E60001D44642394FBF3F6B7FA87FE014603FB27
:108E7000164600F13803019304F0030344604FEAFF
:108E80005E1E00934FF0070C0B7A4A2B0ED14B69F4
:108E9000009AEC1802B906B927B93B2BD4BF0023BE
:108EA000012300E000232344013B3FE0442B02D197
:108EB0004B692B443AE0009B2BB9002E0CBFF046C7
:108EC0004FF0010800E0F046A946244B302202FB97
:108ED0000838CC68A8F1040A0123A34204DA5AF83E
:108EE00004BF0133D944F8E709F1040393FBFCFB09
:108EF000CBEBCB0ACAEB030A4B69012CB8BF0124A8
:108F0000B3EB0A0A0B6904F1804403F1FF3304F167
:108F1000FF3448BF0AF1070AC3EBC30358F82440E3
:108F20005344A34201DB073BFBE74B448C690C4AEB
:108F300002FB03430C6A234441F81C3F019B994206
:108F4000A2D1C369826B9342ACBF002301230360AB
:108F5000012000E0002003B0BDE8F08F60BB0008F6
:108F60008051010070477047014B186800F002B84B
:108F7000240300202DE9F04F8DB0074600F0F8F9EA
:108F8000B0490446384600F0EBF9AF4E054660B9EB
:108F9000AE4BAF4A1860AF4B1860AF4B30681A60E9
:108FA0005A60FFF733FD356048E1316879B93068C0
:108FB000FFF72CFD2846FFF774FE411C3846FFF7EB
:108FC0008DFD306048B12946FFF763FE05E000F0F3
:108FD00081FD002800F03281E9E72B780AAE3A2BB8
:108FE00008BF013533469D4A9D49284600F046FD9D
:108FF000002840F323810A9BEF18EB5C2D2B03D153
:1090000001374FF0FF3503E02B2B08BF0137012557
:109010000DF1200A0DF11E0B4FF000080396CDF85C
:1090200008A00196CDF800B0334607AA8D4938460E
:10903000ADF81E80ADF8208000F020FD404540F3E3
:10904000FD80BDF81E20BDF820303C2101FB02331D
:10905000BDF81C204FF4616101FB02335D437F4B7F
:1090600025627D4DDFF808922B600A9B4A461F441B
:109070007B493346384600F001FD404508DC2B684B
:10908000226A6B60714B1A60724BC3F80080D5E0A6
:109090000A9BC5F80490FD18FB5C2D2B03D101350C
:1090A0004FF0FF3703E02B2B08BF013501270023CA
:1090B000ADF81C30ADF81E30ADF820300A930396A1
:1090C000CDF808A00196CDF800B0334607AA65494F
:1090D000284600F0D3FC002804DC236AA3F5616372
:1090E000E3630EE0BDF81E20BDF820303C2101FBFB
:1090F0000233BDF81C204FF4616101FB02335F4372
:10910000E76327460A9B4FF000091D442B782C2B60
:1091100008BF013595F80080B8F14D0F26D10DF14B
:109120002603029309AB00930396019633460DF193
:1091300022024D49284600F0A1FC03287ED1BDF84B
:1091400022104B1E0B2B79D8BDF82420531E042B64
:1091500074D8BDF82630062B70D887F80880F960DF
:109160003A617B610A9B05EB03082AE0B8F14A0FDC
:1091700006BF4346013544230A220BA9284605931E
:10918000FFF73EFEDDF82C80ADF826004545059B37
:1091900014D14D23B9F1000F07D123720323E360EB
:1091A00002232361C4F814900BE084F824300B23CD
:1091B000A3620123E3620023236302E080B23B72D7
:1091C00078610223ADF81C300023ADF81E30ADF8F5
:1091D00020300A9398F800302F2B0BD10396CDF84E
:1091E00008A00196CDF800B0334607AA1F494046B3
:1091F00000F044FCBDF81E20BDF820303C2101FBEE
:109200000233BDF81C204FF4616101FB0233BB61E6
:109210000A9D09F10109B9F1020F454407F11C0744
:109220007FF474AF6068FFF7F5FD226A074B1A60A0
:10923000E36B9B1A074A18BF012313600DB0BDE80A
:10924000F08F00BFC0BB0008041200200C120020E9
:10925000C3BB00080812002028030020F7110020DB
:10926000C7BB0008EABB0008D6BB0008E9BB000882
:10927000EC11002030B5141E05469BB0184604DAE8
:109280008B232B604FF0FF301DE04FF40273ADF8DD
:109290000C300CBF234604F1FF33029305934FF6C5
:1092A000FF7300910491ADF80E3002461E9B694693
:1092B000284600F053F9431CBCBF8B232B6014B12C
:1092C000009B00221A701BB030BD000007B5009350
:1092D00013460A46014603480068FFF7CBFF03B078
:1092E0005DF804FB240300202DE9F84F07468B4668
:1092F000904600F0F9FB194B1D689A463DB15C465B
:10930000234613F8012B42B13D2A1C46F8D13846BA
:1093100000F0EBFB0020BDE8F88FCBEB0404A9467E
:1093200059F8040B0028F2D022465946FFF7C1FC39
:1093300088B959F8043C1E191B5D3D2B0BD1DAF896
:1093400000303846ED1AAD10C8F8005000F0CDFBE3
:10935000701CBDE8F88F4D46E1E700BF74030020A4
:1093600007B501AAFFF7C0FF03B05DF804FB0000DA
:1093700000487047340300200268464BF0B592FB6A
:10938000F3F403FB1422002ABCBF02F5A83202F555
:10939000C0724FF4616092FBF0F300FB13224FF0B8
:1093A0003C008B6092FBF0F300FB132204F52F24AA
:1093B000ACBF04F66C2404F66B244B600A600723F0
:1093C000E21C92FBF3F3344DC3EBC30394FBF5F5BE
:1093D000D31A48F6AC6240F2B4578B612F4B304839
:1093E00003FB0544B4FBF2F2B4FBF7F3B4FBF0F07B
:1093F0002244D21A48F69466131A40F26D12B3FB57
:10940000F6F6B3FBF2F0B3FBF7F33444E31A02FBD6
:10941000103303EB830299240232B2FBF4F254437B
:10942000A61C0524B6FBF4F40A2A34BF02266FF00A
:10943000090616444FF4C87202FB05055F1C012E95
:1094400098BF0135B3F5997FA7EB040702D3A3F5C5
:10945000997214E0820705D16424B0FBF4F204FB96
:1094600012024AB94FF4C872B0FBF2F402FB1400C6
:10947000B0FA80F2520900E001223B331A44A5F20F
:109480006C750023CA614D610E61CF600B620846A6
:10949000F0BD00BF80510100B13A02004FC5FDFF91
:1094A000B03A0200704770472DE9F0478E68824657
:1094B0009E420C46914698463ED88A8912F4906F97
:1094C0003AD02568096902236F1A656905EB4505DD
:1094D00095FBF3F57B1C43449D4238BF1D46530565
:1094E0000FD52946FFF7FAFA064698B13A462169A0
:1094F000FFF794FAA38923F4906343F08003A381D8
:1095000013E02A4600F01BFB064670B9216950465D
:10951000FFF798FA0C23CAF80030A3894FF0FF3008
:1095200043F04003A381BDE8F08726613E442660F6
:1095300046466561ED1BA560464528BF464649463F
:109540003246206800F0E0FAA36800209B1BA3606D
:1095500023681E442660BDE8F08700002DE9F04F27
:109560009DB003938B8980461C060D4616460DD58B
:109570000B695BB94021FFF7B1FA2860286118B97F
:109580000C23C8F80030CDE040236B610023099321
:1095900020238DF82930DFF89CB130238DF82A3054
:1095A00037463C4614F8013B1BB9B7EB060910D00F
:1095B00003E0252BF9D02746F3E74B4632462946F0
:1095C0004046FFF771FF013000F0A780099B4B4434
:1095D00009933B78002B00F0A08000234FF0FF326E
:1095E00004930793059206938DF853301A9301263E
:1095F000052221784E4800F079FA671C049B38B1A7
:109600004B4A3C46801A06FA00F018430490EFE7F4
:10961000D90644BF20228DF853201A0744BF2B22BD
:109620008DF8532022782A2A03D0079A00210A2095
:109630000BE0039A111D12680391002A10DA5242BE
:1096400043F00200079204900BE027463B78013478
:10965000303B092B03D800FB02320121F5E701B1B1
:1096600007923B782E2B1ED17B782A2B0AD1039BA5
:1096700002371A1D1B680392002BB8BF4FF0FF334F
:10968000059310E0002319460593781C0A24074629
:109690003A780130303A092A03D804FB012101232A
:1096A000F5E703B1059103223978224800F01EFA4C
:1096B00040B14023CBEB000003FA00F0049B0137DC
:1096C00018430490397806221B487E1C8DF8281018
:1096D00000F00CFA88B1194B33B9039B073323F020
:1096E00007030833039314E003AB00932A46144B9B
:1096F00004A94046AFF3008007E003AB00932A467D
:109700000F4B04A9404600F093F8B0F1FF3F8246AA
:1097100003D0099B5344099342E7AB895B0601D40C
:10972000099801E04FF0FF301DB0BDE8F08F00BF99
:10973000FDBC000803BD000807BD000800000000D4
:10974000A99400082DE9F04791461F460A698B68E5
:1097500006469342B8BF1346C9F8003091F843203B
:109760000C46DDF8208012B10133C9F800302368BF
:10977000990642BFD9F800300233C9F80030256895
:1097800015F0060510D104F1190A07E0012352462D
:1097900039463046C04701301AD00135E368D9F860
:1097A00000209B1A9D42F1DB94F84330226800337D
:1097B00018BF012392060FD5E118302081F843002D
:1097C0005A1C94F845102244023382F8431003E0F7
:1097D0004FF0FF30BDE8F08704F1430239463046D0
:1097E000C0470130F4D02268D9F80050E36802F095
:1097F0000602042A08BF5D1B2269A3680CBF25EA84
:10980000E57500259342C4BF9B1AED184FF000097F
:109810001A344D4509D00123224639463046C04707
:109820000130D5D009F10109F3E70020BDE8F08748
:109830002DE9F04317460A7E85B06E2A9846064603
:109840000C460C9B01F1430E00F0AE8011D8632A48
:1098500022D009D8002A00F0BB80582A40F0CA80E4
:1098600081F84520834955E0642A1ED0692A1CD01E
:10987000C0E0732A00F0B08009D86F2A2ED0702A79
:1098800040F0B8800A6842F020020A603EE0752A83
:1098900024D0782A3AD0ADE01A6801F14205111DB2
:1098A0001960136884F84230A8E021681A6811F042
:1098B000800F02D0111D196008E011F0400F02F175
:1098C0000401196002D0B2F9003000E01368002BE7
:1098D0003CDA2D225B4284F8432037E021681A6885
:1098E00011F0800F02D0111D196007E011F0400F38
:1098F00002F10401196001D0138800E01368227E90
:109900005C496F2A14BF0A2208221BE078225A49B8
:1099100084F845202268186812F0800F00F10405D1
:109920001D6003D1550601D5038800E00368D00708
:1099300044BF42F0200222601BB9226822F02002BC
:1099400022601022002084F8430001E049490A22E5
:109950006568002DA56008DB206820F00400206009
:109960002BB9002D7DD175460CE0002B79D07546C2
:10997000B3FBF2F002FB1033CB5C05F8013D03466C
:109980000028F5D1082A0BD12368DA0708D5236906
:1099900062689A42DEBF302305F8013C05F1FF35CD
:1099A000C5EB0E0323612EE008681A6810F0800FE3
:1099B000496903D0101D1860136808E010F0400FCB
:1099C00002F104001860136801D0198000E01960EA
:1099D00000232361754616E01A68111D1960156889
:1099E00000216268284600F081F808B1401B6060E1
:1099F000636804E004F1420584F8422001232361F6
:109A0000002384F84330CDF800803B4603AA21466A
:109A10003046FFF797FE013002D14FF0FF3026E0CD
:109A200023692A4639463046C0470130F5D02368BD
:109A30009B0710D5002504F1190907E001234A46C8
:109A400039463046C0470130E7D00135E368039A14
:109A50009B1A9D42F2DBE068039B9842B8BF184610
:109A600005E00B7804F1420584F842308AE705B03E
:109A7000BDE8F0830EBD00081FBD00080EB430B570
:109A80009CB01FAC4FF4017254F8045BADF8142085
:109A900002900690FFF705F90B4B03900B93002300
:109AA0000F9314934FF6FF7307900848ADF81630E4
:109AB0002A46234602A90068019400F0C1F81CB0B0
:109AC000BDE8304003B07047D19A0008240300205D
:109AD0000020704710F8012B11F8013B012A28BF24
:109AE0009A42F7D0D01A70477047704710B5C9B284
:109AF00002449042034605D01C7801308C42F8D1D4
:109B0000184610BD002010BD884210B501EB0203BD
:109B100001D8421E0BE09842FBD28118D21AD342E0
:109B200004D013F8014D01F8014DF8E710BD99423A
:109B300004D011F8014B02F8014FF8E710BDF8B559
:109B4000074615460E4621B91146BDE8F840FEF716
:109B5000C5BF1AB9FEF776FF2846F8BD00F00BFC2A
:109B600085420ED929463846FEF7B8FF044650B163
:109B700031462A46FEF752FF31463846FEF762FF6D
:109B800001E03046F8BD2046F8BD4B1C70B50E46CE
:109B9000144602D14FF0FF3070BD9389CDB223F04F
:109BA00020039381536B526883B1A36B9A4207DA07
:109BB00023685A1E226003F8016C636801331FE0BA
:109BC000214600F09FFB0028F2D0E3E721692368DB
:109BD00051B1994208D213F8011C8D4204D1013BC6
:109BE0000132236062600CE0E36304F144036363C9
:109BF0000323A3632346226403F8466F23600123F3
:109C00006360284670BD10B50C46496B69B104F11C
:109C10004403994201D0FEF715FF236C00206063D6
:109C2000636013B1E36B236010BD23694FF0FF3015
:109C3000236000236360A38943F02003A38110BD48
:109C40002DE9F04FDFF89C9207460D46CA46ADF568
:109C5000257D01930023469347939E4B0DF10C08FD
:109C6000A2939D4BDFF874B2CDF82081A3931478B2
:109C7000002C00F02781D9F8003023445B7803F0F2
:109C8000080303F0FF01F3B16B68002B10DD2B68B4
:109C9000DAF800001978014449780C0710D5479983
:109CA00001330131479169682B6001396960EBE745
:109CB000A39B2946384600929847009A0028E6D090
:109CC000561C3246D3E7252C02F1010652D14391AE
:109CD000459153782A2B02BF1023961C43930A22E6
:109CE00031783446A1F13003092B06F1010605D87D
:109CF000459B02FB0313303B4593F1E70322774872
:109D0000FFF7F4FE40B134460123CBEB000003FA29
:109D100000F0439B03434393661C2478672C16D8BA
:109D2000652C7FD2472C07D8452C7BD2002C00F025
:109D3000CB80252C1ED077E05B2C51D002D8582C3C
:109D40003ED071E0632C57D0642C3FD06CE0702C77
:109D500032D007D86E2C55D03AD8692C64D1002364
:109D600044933BE0752C31D0782C29D0732C5BD1F7
:109D700002233FE06B68002B0DDD2B681A789442BC
:109D800040F0A08001336A682B60479B013A0133A1
:109D90006A60479395E7A39B294638469847002871
:109DA000EBD04698002800F08F80AB8913F0400F6D
:109DB00018BF4FF0FF3089E0439B43F020034393EB
:109DC000439B43F400734393102302E00A2300E013
:109DD00008236E2C449301DD04230BE0032309E0E8
:109DE0003146404600F0D8F90646439B43F0400315
:109DF0004393012349931BE0439B43F04003439368
:109E00000023F7E7439AD0063FF55BAF12F0010F4E
:109E1000019A479B02F104010191126814BF13805B
:109E200013604EE70523E5E7032349930A23449390
:109E30006B68002B03DD439B590611D518E0A39BEB
:109E40002946384698470028F5D0AAE7479A0132B4
:109E500047926A68013A002A6A6013DD01332B6079
:109E60002B68DAF800101A780A4452781207EDD4F9
:109E7000499B022B0DDC01AB2A4643A9384600F072
:109E800033F819E0A39B2946384698470028E7D0C5
:109E900087E7042B06DC01AB2A4643A9384600F0CD
:109EA00089F809E00E4B002B3FF40BAF01AB2A46BB
:109EB00043A93846AFF30080012803D002287FF47D
:109EC00000AF6EE7469801E04FF0FF300DF5257DBD
:109ED000BDE8F08F8B9B0008079C000803BD0008BD
:109EE00000000000300300202DE9F84315468A6881
:109EF00080460C4632B98A69002A0CBF01224FF015
:109F0000FF328A602268DFF8A890D10658BF1A682D
:109F10004FF000065EBF111D19601768A069F8B9FF
:109F200023680136DA065EBF2B681B783B702A680F
:109F30006B6802F101022A60A26803F1FF3302F1AB
:109F4000FF326B6058BF0137A260E2B1002BE5DC45
:109F5000D4F880312946404698470028DED012E0E8
:109F6000012806D12B681A7863699B5C002BD7D136
:109F700019E0022807D12B68D9F800201B78134478
:109F80005B781B07CCD5236813F0100305D1E2687A
:109F90000132E260A26902B13B70236900201E44D5
:109FA0002661BDE8F883002EEDD1BDE8F88300BF3F
:109FB000300300202DE9F04F0C469A46724B87B0D3
:109FC0008346164693E8070003ABA76883E80700BB
:109FD0006E4BA1696E4A04F11C09032918BF1A4689
:109FE0007B1EB3F5AE7F84BF40F25D13A360236890
:109FF00088BF6FF4AE7543F4506323604B46009204
:10A000008CBF7F1900274FF000083168019303AB24
:10A0100053F8280002220978FFF768FD019B002809
:10A0200033D0B8F1010F0BD162682AB908226260FF
:10A03000226842F400722260226822F4A0620CE0DE
:10A04000B8F1020F0AD1226802F4C061B1F5007FB5
:10A050001BD11021616042F480722260A268511EFF
:10A06000A16092B132685D1C511C316012781A7087
:10A070007368013B002B736006DCD4F880313146F5
:10A0800058469847002841D12B4608F10108B8F1FD
:10A09000030FBAD162680AB90A22626062683D4958
:10A0A0006069891A019300F077F8019B4FF000086E
:10A0B0001D46A36863B3316860690A78805C38B371
:10A0C000302A226808D1100506D508F1010857B1D9
:10A0D0000133013FA36006E022F4106222600B7896
:10A0E000013505F8013C7368013B002B736003DD0B
:10A0F00033680133336005E0D4F880313146584687
:10A10000984728B9A368013BA360D2E74FF0000845
:10A110002368D9050CD54D4508D915F8011C6F1ECB
:10A12000D4F87C313246584698473D464D4527D0B5
:10A13000226812F010021BD12A7063684946584603
:10A14000009EB0472268DAF8003012F0200F07D1E5
:10A15000D20705D51A1DCAF800201B68188004E034
:10A160001A1DCAF800201B681860E3680133E36019
:10A170002369C9EB050545441D442561002000E025
:10A18000012007B0BDE8F08F30BD0008058D000844
:10A19000F9A100084CBD000870B50B78441E5E2B79
:10A1A00013BF4A1C8A1C4B78002108BF012100F113
:10A1B000FF0504F8011FAC42FBD10BB9501E70BD66
:10A1C00081F001041146C4540D784A1C2D2D06D08F
:10A1D0005D2D0FD00DB12B46F4E7084670BD4E78CB
:10A1E0005D2EF8D0B342F6DC023101339E42C454F6
:10A1F000FBDCE9E7104670BD2DE9F0470F468046CD
:10A200003F48D0F800903D4615F8014B09EB04009B
:10A21000407800F0080000F0FF0608B12F46F2E792
:10A220002D2C03D1BD1C7C78012603E02B2C04BF10
:10A230007C78BD1C13B1102B0AD15BE0302C57D1B8
:10A24000287800F0DF0058284DD16C7810230235B3
:10A25000002E14BF4FF0004C6FF0004CBCFBF3FA23
:10A260000027384603FB1ACC09EB040E9EF801E0E8
:10A270001EF0040F01D0303C0BE01EF0030E1BD08B
:10A28000BEF1010F0CBF4FF0370E4FF0570ECEEB63
:10A290000404A34210DDB7F1FF3F0AD0504506D8B1
:10A2A00001D1644503DC03FB0040012701E04FF0CE
:10A2B000FF3715F8014BD7E77B1C0CD1002E4FF070
:10A2C000220314BF4FF000406FF00040C8F8003088
:10A2D0002AB9BDE8F08706B1404272B107B1691EE4
:10A2E0001160BDE8F0873024002BB1D10823AFE71F
:10A2F0000A23ADE7302CA3D0AAE7BDE8F08700BF62
:10A30000300300202DE9F0410C46496B04F1440371
:10A3100099421AD14FF48061FEF7E0FB18B94FF073
:10A32000FF30BDE8F0814FF48063A36394F84630BA
:10A33000606380F8FF3394F8453000F2FD304370DD
:10A3400094F844300370206012E0A66B77003A4620
:10A35000FFF7F5FB05460028E1D000EB06080146B3
:10A3600032464046FEF75AFBC4F800806563A76397
:10A370000020BDE8F08151F8040C0028BEBF091888
:10A3800051F8043CC018043870470000044B0246E2
:10A39000196809B903491960186802441A607047BE
:10A3A00014120020A0140020FEE70000F8B500BF42
:10A3B000F8BC08BC9E467047F8B500BFF8BC08BCA6
:10A3C0009E46704765617374657220646174653A76
:10A3D00020253034642D253032642D253032640D33
:10A3E0000A00536F004D6F004469004D6900446FCF
:10A3F00000467200536100537500547500576500A4
:10A400005468004443463737204572726F723A20D1
:10A41000486967682070756C7365203C3D20350085
:10A420004443463737204572726F723A2048696755
:10A43000682070756C7365203E3D203235004443C2
:10A44000463737204572726F723A207061726974B4
:10A450007920503120696E636F72726563740044B5
:10A4600043463737204572726F723A2070617269C5
:10A47000747920503220696E636F72726563740064
:10A480004443463737204572726F723A20706172CA
:10A4900069747920503320696E636F7272656374DA
:10A4A00000003F3F0A0000000B00000057A5000815
:10A4B000C6A500080A0000000B00000035A6000831
:10A4C000A4A600080A0000000B00000013A7000863
:10A4D00082A7000800000100010002000200030042
:10A4E0000300040004000500050006000700080042
:10A4F00009000B000D000E001000120014001700E0
:10A5000019001C001F002100240028002B002E0031
:10A510003200360039003D00420046004A004F003C
:10A52000540059005E00630069006E0074007A00F8
:10A53000800086008C0093009900A000A700AE0068
:10A54000B600BD00C500CD00D500DD00E500EE0081
:10A55000F600FF00257500303030303030303030BC
:10A5600030303030313131303131313030303131E3
:10A5700031313131313131303131313131313131CC
:10A5800031313131313131313131313131313031BC
:10A5900031313131313131313030303131313131AE
:10A5A00031313030303030313131313130303030A4
:10A5B0003030303131313030303030303030303197
:10A5C00030303030300030303030303030303030BB
:10A5D00030303045454530454545303030464544BE
:10A5E0004343434445313047464443424242434457
:10A5F0004647474644434241424344464730464427
:10A60000434242424344463030304544434343444E
:10A6100045303030303045444444313030303030D3
:10A6200030304545453030303030303030304630D5
:10A630003030303000303030303032303030303048
:10A6400030303033323232333030303030303231FB
:10A6500032313230303030333232323232323233E1
:10A6600030303232313232323132323030303232D6
:10A6700032323232323030333231323232323231BF
:10A6800032333232323232323232323232303030AF
:10A69000303838383030303030303030383838308A
:10A6A00030303000303030303041303030303030C9
:10A6B00030305441414154303030303030414A41E3
:10A6C0004A413030303054414141414141415430A0
:10A6D0003041414A4141414A41413030304141419C
:10A6E00041414141303054414A41414141414A4157
:10A6F000544141414141414141414141303030307B
:10A7000041414130303030303030304141413030E3
:10A710003030003030303036303031303030303161
:10A72000313033303130313031313030313031301F
:10A730003031303030353030313031303030303011
:10A7400030313330373030353130303030333733EB
:10A7500030303630303030303037303030303030EC
:10A7600030303037303030303030303030303730DB
:10A7700030303030303030303037303030303030D2
:10A780003000303030305030304B303030304C4B87
:10A7900030503049304A304B4D30304830483030FE
:10A7A0004830303050303047304730303030303043
:10A7B000494830463030504A3030303049454930D1
:10A7C000304830303030303044303030303030305D
:10A7D0003030433030303030303030303042303054
:10A7E0003030303030303030413030303030303058
:10A7F000004E6F6E65004661646500526F6C6C00C0
:10A800004578706C6F64650052616E646F6D0053C3
:10A810006E616B650054656C657479706500437595
:10A820006265004D61747269780044726F70005304
:10A83000717565657A6500466C69636B6572005277
:10A8400061696E626F77004E6F726D616C00436C70
:10A850006F636B00436C6F636B320000000000009D
:10A860000000000C12120C000000000A00040A1183
:10A870001F1100120C121212120C000A00121212F6
:10A88000120C000A000E010F110F000A000C121228
:10A89000120C001200121212160A00001C121C12D6
:10A8A000121C10000000000000000000000000006A
:10A8B0000000000000000000000000000000000098
:10A8C0000000000000000000000000000000000088
:10A8D0000000000000000000000000000000000078
:10A8E0000000000000000000000000000000000068
:10A8F0000000000000000000000000000000000058
:10A900000000000000000000000000000000000047
:10A910000000000000000000000000000000000037
:10A920000000000000000000000000000000000027
:10A930000000000000000000000000000000000017
:10A940000000000000000000000000000000000007
:10A9500000000000000000000000000000000000F7
:10A96000000000040E0E04040004001B1B12000073
:10A97000000000000A1F0A0A1F0A00080E100C023D
:10A980001C040019190204081313000814140815F4
:10A99000120D000C0C080000000000040808080854
:10A9A0000804000804040404040800000A0E1F0E32
:10A9B0000A00000004041F0404000000000000005E
:10A9C0000C0C080000001F00000000000000000048
:10A9D0000C0C0000010204081000000E11131519E0
:10A9E000110E00040C040404040E000E11010608EC
:10A9F000101F000E11010E01110E0002060A121F97
:10AA00000202001F10101E01110E000608101E1178
:10AA1000110E001F010204080808000E11110E118A
:10AA2000110E000E11110F01020C0000000C0C00A1
:10AA30000C0C0000000C0C000C0C080204081008A0
:10AA400004020000001F00001F00000804020102B1
:10AA50000408000E110106040004000E111715175A
:10AA6000100E000E1111111F1111001E11111E11D7
:10AA7000111E000E11101010110E001E11111111D7
:10AA8000111E001F10101E10101F001F10101E108E
:10AA90001010000E11101711110F001111111F11BC
:10AAA0001111000E04040404040E0001010101113F
:10AAB000110E0011121418141211001010101010A1
:10AAC000101F00111B15111111110011191513116F
:10AAD0001111000E11111111110E001E11111E1075
:10AAE0001010000E11111115120D001E11111E1261
:10AAF0001111000E11100E01110E001F04040404A8
:10AB00000404001111111111110E00111111111174
:10AB10000A04001111151515150A0011110A040A6D
:10AB20001111001111110A040404001E020408107E
:10AB3000101E000E08080808080E00001008040285
:10AB40000100000E02020202020E00040A110000BF
:10AB5000000000000000000000003F0C0C0400009A
:10AB600000000000000E010F110F0010101E111147
:10AB7000111E0000000E1110110E0001010F111125
:10AB8000110F0000000E111E100E000608081E080E
:10AB900008080000000F11110F010E10101C1212F6
:10ABA000121200040004040404060002000602025B
:10ABB00002120C10101214181412000404040404DD
:10ABC00004060000001A151511110000001C1212D5
:10ABD00012120000000E1111110E0000001E1111C2
:10ABE000111E1000000F1111110F010000160908AD
:10ABF000081C0000000E100E010E0000081E0808C0
:10AC00000A04000000121212160A000000111111AD
:10AC10000A040000001111151F0A00000012120C96
:10AC200012120000001212120E041800001E020C74
:10AC3000101E000608081808080600040404000492
:10AC40000404000C02020302020C000A14000000BB
:10AC500000000000000000000000000000003F00B5
:10AC600000003F003F3F0000003F3F003F003F3FEC
:10AC70003F3F3F20200020202001021B1C474800AE
:10AC800000000000000100030A00000100040A00A7
:10AC9000000100080A00000104040B0C0001040379
:10ACA0000B0C0001040C0000000104030A0C00015D
:10ACB00004040A0C000104080B00000104040B004A
:10ACC000000104030B00000000000000000100036D
:10ACD0000A00000100040A0000010408000000014D
:10ACE00004040B0C000104030B0C0001040C000015
:10ACF000000104030A0C000104040A0C0001040909
:10AD00000000000104040B00000104030B0000001C
:10AD100000000000000100030A00000100040A0016
:10AD2000000100080A00000100050A0000010403F8
:10AD30000B0C0001040C0000000104030A0C0001CC
:10AD400004050B00000104080B00000104040B00C3
:10AD5000000104030B0000000000000000010003DC
:10AD60000A00000100040A000001040800000001BC
:10AD700000050A00000104030B0C0001040C000094
:10AD8000000104030A0C000104050B000001040982
:10AD90000000000104040B00000104030B0000028A
:10ADA000010000000003011D22000003011F22001A
:10ADB0000003011E22000003012022000003051DE4
:10ADC00021230003052300000003051D22230003A7
:10ADD000052021000003051E21000003051F21009E
:10ADE0000003051D210000040100000000050133DF
:10ADF0003800000501353800000501343800000531
:10AE000001363800000505333739000505390000E3
:10AE100000050533383900050536370000050534CF
:10AE200037000005053537000005053337000006FB
:10AE3000020000000007024D51000007024F5100C0
:10AE40000007024B51000007024C51000007024C62
:10AE50004D510007024E00000007064C4D50000700
:10AE6000064C50000007064B50000007064F5000EC
:10AE70000007064D500000080200000000090263B0
:10AE800067000009026567000009026167000009A8
:10AE90000262670000090262636700090264000041
:10AEA0000009066263660009066266000009066121
:10AEB0006600000906656600000906636600005723
:10AEC00045535349004F53534900524845494E2D6D
:10AED0005255485200534348574142454E00534350
:10AEE000485745495A4552444555545343482031E3
:10AEF000005343485745495A4552444555545343D6
:10AF000048203200454E474C4953434820310045C4
:10AF10004E474C49534348203200000000000002D5
:10AF200000030300070401000401040702000402F7
:10AF3000040402040702000B0302040306030400D6
:10AF400004040505050004050203050204050506C1
:10AF500006010406070407000307030407070408A3
:10AF600001040805040901050908030000020003A3
:10AF7000040008030100060108030200060208039A
:10AF8000030002030305040003040304040803058B
:10AF90000005050504060006060605070005070569
:10AFA0000408000408070409000609080300000259
:10AFB0000003040100040105060008030200060264
:10AFC0000803030002030305040003040304040848
:10AFD000030500050506050600060606050700052B
:10AFE000070604080004080704090006090803000E
:10AFF000000200030200070200090201020702002A
:10B000000602060403000403050303090204000406
:10B0100004070405000305030305060506000406EE
:10B0200004040608030700050705060800050805CF
:10B0300006090003090506000002000302010407D7
:10B0400002010602070400060401000303000203D4
:10B0500002040407040607030804030500050307A8
:10B06000040400040404030706050601060700059E
:10B070000505060801030904010906050D1A000F5C
:10B080001A000E1A00121A00161A00131A00191AC2
:10B0900000111A00171A00151A00181A00141A00C5
:10B0A0000D00001000000E0000120000160000133A
:10B0B0000000190000110000170000150000180022
:10B0C000001400002F30002430002530002630000E
:10B0D0002730002830002930002A30002B30002C87
:10B0E00030002D30002E30002F00002400002500FD
:10B0F000002600002700002800002900002A000088
:10B100002B00002C00002D00002E00004500003A0E
:10B1100000003B00003C00003D00003E00003F00FE
:10B1200000400000410000420000430000440000D5
:10B130004500003A00003B00003C00003D00003E9E
:10B1400000003F00004000004100004200004300BA
:10B15000004400005C5E00535E00585E00555E00D7
:10B16000565E00575E00545E005B5E00595E005202
:10B170005E005D5E005A5E005C00005300005800F7
:10B18000005500005600005700005400005B00000E
:10B190005900005200005D00005A00007274756989
:10B1A00074756E74756B74756C74756D74756A7482
:10B1B000757174756F747568747573747570747562
:10B1C0007200006900006E00006B00006C00006DF2
:10B1D00000006A00007100006F000068000073004A
:10B1E000007000002800290D0A004F4B0045525204
:10B1F0004F52002D200049504144445245535320A2
:10B2000000415020004D4F444520006170005449DA
:10B210004D4520005745415448455220004649526B
:10B220004D574152452000434D4420002D2D3E20D6
:10B23000003C253032783E003C30643E3C30613E7C
:10B240000D0A0063617020222573222C22257322AF
:10B25000007770730045535038323636204C4F47D4
:10B260004745520D0A000000010000000F000000D9
:10B2700015000000070000000B00000007000000A0
:10B280000B000000070000000B0000000F00000092
:10B2900014000000000000000F0000001400000077
:10B2A000000000000100000000000000020000009B
:10B2B000050000000C00000011000000220000004A
:10B2C000050000000C000000050000000C0000005C
:10B2D000000000000000000000000000000000006E
:10B2E000000000000100000001000000000000005C
:10B2F00005000000020000000B0000000C00000030
:10B300001A000000020000000B0000000200000014
:10B310000B00000000000000100000001C000000F6
:10B3200028000000300000000100000001000000C3
:10B330000000000002000000050000000C000000FA
:10B340001100000022000000050000000C000000B9
:10B35000050000000C0000000000000010000000CC
:10B36000100000002000000020000000010000008C
:10B3700001000000000000000300000005000000C4
:10B380000C0000000F0000001E000000050000007F
:10B390000C000000040000000B0000000000000092
:10B3A000100000001500000025000000250000002E
:10B3B00001000000010000000000000057726974E5
:10B3C000696E6720257320746F20454550524F4D9C
:10B3D000206661696C65640D0A002E35000D0A5700
:10B3E000656C636F6D6520746F20576F7264436C7A
:10B3F0006F636B204C6F6767657221002D2D2D2DBB
:10B400002D2D2D2D2D2D2D2D2D2D2D2D2D2D2D2D6C
:10B410002D2D2D2D2D2D2D2D0056657273696F6EDE
:10B420003A2000322E362E34007274632069732065
:10B430006F6E6C696E6500727463206973206F664D
:10B44000666C696E6500656570726F6D206973204A
:10B450006F6E6C696E650063757272656E742065DF
:10B460006570726F6D2076657273696F6E3A203009
:10B4700078253038780D0A0075636C6F636B2E6425
:10B48000650075706461746500656570726F6D202C
:10B490006973206F66666C696E65007570646174AF
:10B4A000696E6720454550524F4D20746F20766578
:10B4B0007273696F6E203078253038780D0A007607
:10B4C000657273696F6E00495220636F6465730023
:10B4D000646973706C617920636F6E6669677572F9
:10B4E0006174696F6E0074696D65736572766572FB
:10B4F00020636F6E66696775726174696F6E006E46
:10B50000696768742074696D6520636F6E6669672A
:10B5100075726174696F6E0074656D7065726174C7
:10B5200075726520636F6E66696775726174696FA5
:10B530006E0052544320636F6E6669677572617462
:10B54000696F6E004C445220636F6E666967757256
:10B550006174696F6E007765617468657220636FEE
:10B560006E66696775726174696F6E007573657276
:10B5700020627574746F6E20707265737365643ABF
:10B5800020636F6E6669677572696E672065737098
:10B5900038323636206173206163636573732070BF
:10B5A0006F696E74003132333435363738393000D4
:10B5B000776F7264636C6F636B0077707320627572
:10B5C00074746F6E20707265737365643A2073656E
:10B5D0006E64696E67206573703832363620777016
:10B5E0007320636F6D6D616E640049502025730098
:10B5F000696E666F3A206970206164647265737366
:10B60000203D2025730D0A00696E666F3A2077652C
:10B610006174686572203D2025730D0A00657370A2
:10B6200038323636206E6F7720757000657370384B
:10B63000323636206E6F77206F6E6C696E650064EF
:10B64000636637373A202573202534642D25303240
:10B65000642D2530326420253032643A253032643E
:10B660003A253032640D0A00726561642072746399
:10B670003A202573202534642D253032642D253061
:10B68000326420253032643A253032643A25303233
:10B69000640D0A00466F756E642054696D65723AD8
:10B6A00020257320617420253032643A25303264BD
:10B6B0000D0A00466F756E642054696D65723A20FC
:10B6C000616D62696C6967687420257320617420FC
:10B6D000253032643A253032640D0A004453313843
:10B6E0007878782074656D70657261747572653AEA
:10B6F00020256425730D0A005254432074656D7033
:10B70000657261747572653A20256425730D0A00AF
:10B7100069636F6E3A2025640D0A0073686F7720A5
:10B7200064617465206173207469636B65720025C0
:10B730003032642E253032642E25640075706461C9
:10B740007465206D61696E20706172616D657465EC
:10B75000727320636F6E66696775726174696F6E6C
:10B7600000706F7765725F696E6974282920636164
:10B770006C6C656400737769746368696E672070C8
:10B780006F776572206F6E00737769746368696E96
:10B790006720706F776572206F666600676574203A
:10B7A00074656D706572617475726500746F67673A
:10B7B0006C65206175746F206272696768746E656C
:10B7C0007373006F6B0064656372656D656E7420E2
:10B7D000646973706C6179206D6F646500696E6374
:10B7E00072656D656E7420646973706C6179206D2B
:10B7F0006F64650064656372656D656E7420616E6B
:10B80000696D6174696F6E206D6F646500696E6348
:10B8100072656D656E7420616E696D6174696F6EBD
:10B82000206D6F64650064656372656D656E74207C
:10B83000686F757200696E6372656D656E742068FD
:10B840006F75720064656372656D656E74206D69F5
:10B850006E75746500696E6372656D656E74206DDA
:10B86000696E7574650064656372656D656E7420DC
:10B87000726564206272696768746E6573730069CB
:10B880006E6372656D656E742072656420627269A4
:10B890006768746E6573730064656372656D656E69
:10B8A0007420677265656E206272696768746E6580
:10B8B000737300696E6372656D656E74206772657F
:10B8C000656E206272696768746E65737300646583
:10B8D0006372656D656E7420626C75652062726955
:10B8E0006768746E65737300696E6372656D656E0B
:10B8F0007420626C7565206272696768746E657326
:10B90000730064656372656D656E7420676C6F6249
:10B91000616C206272696768746E65737300696E2A
:10B920006372656D656E7420676C6F62616C206216
:10B9300072696768746E65737300706F77657220E3
:10B940006F66662F6F6E0020205468616E6B2079E1
:10B950006F752100003F3F00003F2020203F3F0047
:10B96000003F003F003F3F0000000F0000020202C6
:10B970000200000F0004040404080E000006040482
:10B9800000000E020004040C00020E000004040675
:10B9900000000E08000C0404000606000006060065
:10B9A000000606000006060000060C000004060261
:10B9B0000000060C00080C0400040E00000406043D
:10B9C00000000E0400040C04000C06000002060433
:10B9D00000000C0600040C08003F3F3F50756E6BE2
:10B9E00074653A20256C64003139322E35332E319E
:10B9F00030332E313033004E65772074696D657AAF
:10BA00006F6E653A2025640D0A0074696D65202209
:10BA10002573220074696D6500766172200076617D
:10BA2000725F73656E645F6275663A2065787065F3
:10BA30006374656420455350383236365F4F4B2C63
:10BA400020676F742025640D0A0044432530327846
:10BA50002530327825303278253032783030002564
:10BA600073253032782573002573253032782530E0
:10BA70003278004E253032782530327825303278D1
:10BA80000053253032782573005425303278253024
:10BA900034642530326425303264253032642530F8
:10BAA00032642530326400444E25303278257300EC
:10BAB000414E00414400414500414600434E004391
:10BAC00044004345004346004D4E004D44004D4563
:10BAD000004D4600742530327825303278253032DA
:10BAE000782530327800612530327825303278255B
:10BAF00030327825303278006E2530327825303279
:10BB0000782530327800776561746865722022008C
:10BB1000222C22007773323831323A2065787465EE
:10BB2000726E616C2070756C6C75702064657465E4
:10BB300063746564007773323831323A206E6F2057
:10BB400065787465726E616C2070756C6C757020B0
:10BB5000646574656374656400430000C40200207A
:10BB60001F0000001C0000001F0000001E0000005D
:10BB70001F0000001E0000001F0000001F0000004A
:10BB80001E0000001F0000001E0000001F0000003B
:10BB90001F0000001D0000001F0000001E0000002C
:10BBA0001F0000001E0000001F0000001F0000001A
:10BBB0001E0000001F0000001E0000001F0000000B
:10BBC000545A00474D54002531305B5E302D392CDE
:10BBD0002B2D5D256E004D256875256E2E2568750B
:10BBE000256E2E256875256E002F256875256E3A01
:10BBF000256875256E3A256875256E000020202081
:10BC0000202020202020282828282820202020200C
:10BC100020202020202020202020202020881010DC
:10BC20001010101010101010101010101004040438
:10BC300004040404040404101010101010104141F6
:10BC400041414141010101010101010101010101E4
:10BC500001010101010101011010101010104242F8
:10BC600042424242020202020202020202020202B4
:10BC70000202020202020202101010102000000054
:10BC800000000000000000000000000000000000B4
:10BC900000000000000000000000000000000000A4
:10BCA0000000000000000000000000000000000094
:10BCB0000000000000000000000000000000000084
:10BCC0000000000000000000000000000000000074
:10BCD0000000000000000000000000000000000064
:10BCE0000000000000000000000000000000000054
:10BCF00000000000000000000000000000232D30C4
:10BD00002B2000686C4C0065666745464700303163
:10BD100032333435363738394142434445460030B2
:10BD200031323334353637383961626364656600E1
:10BD30004EBD00087FA7000851BD0008412D466197
:10BD40002D66383930313233343536375D002B2D9E
:10BD50000078580000000000000000000000000013
:10BD600000000000000000000000000000000000D3
:10BD700000000000000000000000000000000000C3
:10BD800000000000000000000000000000000000B3
:10BD900000000000000000000000000000000000A3
:10BDA0000000000000000000000000000000000093
:08BDB00000000000000000008B
:08BDB8009043FF7F0100000031
:10BDC000F7A30008E5A30008FAA30008FDA30008F4
:10BDD00000A40008F1A30008F4A30008FF0000007D
:10BDE000FF0000000A0000006400000020000000C6
:10BDF0000000000000000000000000000F00000034
:10BE00000F0000000000000003000000010000001F
:10BE10000000000000000000010000000100000020
:10BE2000FF00000000000000000001FF02FF000012
:10BE3000160000003C000000200000200000000070
:10BE4000F1A70008051C0008040000000400000021
:10BE500000000000F6A700087D190008040000009B
:10BE60000400000003000000FBA700080D170008F5
:10BE700004000000040000000300000000A8000807
:10BE8000191500080600000006000000030000006D
:10BE900008A80008890D0008040000000400000044
:10BEA000000000000FA80008791E00080400000030
:10BEB000040000000300000015A800088114000819
:10BEC0000400000004000000030000001EA8000899
:10BED000211300080400000004000000030000001B
:10BEE00023A80008B11C00080400000004000000A2
:10BEF000030000002AA800081D110008040000002B
:10BF000004000000030000002FA80008291000080A
:10BF100004000000040000000300000037A800082F
:10BF2000B90F000804000000040000000300000036
:10BF3000F1A700080100000001000000000000005F
:10BF40003FA80008040000000400000001000000F9
:10BF500047A80008000000000000000000000000EA
:10BF60004EA80008000000000000000000000000D3
:10BF700054A80008000000000000000000000000BD
:10BF80003FA80008040000000400000001000000B9
:10BF9000080000000800000009000000090000007F
:10BFA0000A0000000A0000000B0000000B00000067
:10BFB0000C0000000C0000000D0000000D0000004F
:10BFC0000E0000000E0000000F0000000F00000037
:10BFD0000300000020000000050000000500000034
:10BFE000EC030020FF000000BFAE0008C5AE000853
:10BFF000CAAE0008D5AE0008DEAE0008F1AE0008FB
:10C0000004AF00080FAF0008FFFF0000FFFF0000B3
:10C01000D80E0000FFFF0000FF000000FFFFFFFF41
:10C02000FF000000FF000000000000000000000012
:10C03000FF00000000000000FF00000004030303F5
:10C04000030303003139322E35332E3130332E3194
:10C050003033000000000000010000000204060868
:10C06000000000000102030401020304060708099E
:10C070000000000000000000010203040607080998
:10C0800000A24A040000000054BD000874BD00086E
:10C0900094BD000800000000000000000000000047
:10C0A0000000000059BB0008000000000000000074
:10C0B0000000000000000000000000000000000080
:10C0C0000000000000000000000000000000000070
:10C0D0000000000000000000000000000000000060
:10C0E00000000000C4020020C3BB0008C3BB00085E
:10C0F000FCBB000801000000000000004A00000036
:10C10000000000000000000000000000000000002F
:10C1100000000000000000004A00000000000000D5
:10C12000000000000000000000000000000000000F
:10C13000000000001012002011010008ED000008AE
:0400000508000000EF
:00000001FF
